:100000002BC3000048C3000046C3000044C30000E7
:1000100042C3000040C300003EC300003CC30000D8
:100020003AC3000038C3000036C3000034C30000E8
:100030000C94CD3E30C300002EC300002CC3000042
:100040002AC3000028C300000C94B93E24C300005A
:1000500022C3000020C300001EC300001CC3000018
:100060001AC3000018C3000016C3000014C3000028
:1000700012C3000010C300000EC300000CC3000038
:100080000AC3000008C3000006C30000510F980F08
:10009000C80FF80F50106B109B10D2103B110211BB
:1000A000760F7B0FCD10F710FC10890F8E0F930F7A
:1000B00088139313951397139A139D13B713B913BA
:1000C000C613D213D516DA16E816ED16F216F71681
:1000D000FC160117951B981B9B1B9E1BA11BA41BA9
:1000E000A71BAA1B78259D25B125C425C725D82582
:1000F000E92507268E259125FA25FD25002694253C
:1001000097259A25042B092B0E2B132B182B1D2B0F
:10011000222B272B2C2B2F2BE32C4E2D722EDB2E5C
:10012000FA2F26310C32013330347F34E2342C354F
:1001300033358735DC35DF35E235E535E835EB3508
:10014000EE35F1358D38A338B938D038E638FC387B
:10015000123928397C397F398239853988398B3988
:100160008E399139CB39E039F539083A1B3A293AB9
:100170003C3A4F3A623A773A8C3AA13AC03AD93A85
:10018000000000000000000004040404000400005B
:100190000A0A0A00000000000A0A1F0A1F0A0A00D1
:1001A000040F140E051E040018190204081303009E
:1001B0000C12140814120D000C04080000000000BA
:1001C00002040808080402000804020202040800ED
:1001D0000004150E150400000004041F04040000B0
:1001E000000000000C0408000000001F00000000D8
:1001F00000000000000C0C000001020408100000C8
:100200000E11131519110E00040C040404040E0041
:100210000E11010204081F001F02040201110E004A
:1002200002060A121F0202001F101E0101110E0019
:100230000608101E11110E001F0102040808080014
:100240000E11110E11110E000E11110F01020C00F2
:100250000001020408100000000C0C000C0408004F
:10026000020408100804020000001F001F00000024
:1002700008040201020408000E1101020400040037
:100280000E11010D15150E000E1111111F11110087
:100290001E11111E11111E000E11101010110E0052
:1002A0001C12111111121C001F10101E10101F0023
:1002B0001F10101E101010000E11101711110E003B
:1002C0001111111F111111000E04040404040E0079
:1002D0000702020202120C0011121418141211006B
:1002E0001010101010101F00111B15151111110006
:1002F00011111915131111000E11111111110E0008
:100300001E11111E101010000E11111115120D00EA
:100310001E11111E141211000F10100E01011E00EB
:100320001F040404040404001111111111110E0022
:1003300011111111110A04001111111115150E00DE
:1003400011110A040A1111001111110A0404040008
:100350001F01020408101F000E08080808080E00FC
:10036000110A1F041F0404000E02020202020E0002
:10037000040A1100000000000000000000001F003F
:10038000080400000000000000000E010F110F0023
:1003900010101E1111111E0000000E1010110E0081
:1003A00001010D1311110F0000000E111F100E009E
:1003B0000609081C08080800000F11110F010E00A3
:1003C000101016191111110004000C0404040E0081
:1003D0000200060202120C0010101214181412006F
:1003E0001808080808081C0000001A15151111004B
:1003F000000016191111110000000E1111110E004C
:1004000000001E111E10100000000F110F0101004E
:10041000000016191010100000000E100E011E0032
:1004200008081C08080906000000111111130D002E
:1004300000001111110A04000000111111150A0029
:100440000000110A040A1100000011110F010E0032
:1004500000001F0204081F00384444447C44440048
:100460007C404078444478007844447844447800A0
:100470007C404040404040000C14242424243C4450
:100480007C40407840407C005454543854545400CC
:10049000384404180444380044444C546444440030
:1004A00054444C5464444400444850605048440010
:1004B0001C24242424246400446C545444444400E4
:1004C0004444447C44444400384444444444380054
:1004D0007C444444444444007844447840404000D0
:1004E00038444040404438007C1010101010100078
:1004F0004444443C044438003854545438101000E8
:1005000044442810284444004444444444447E0263
:10051000444444443C0404005454545454547C0013
:100520005454545454547E026020203824243800FB
:100530004444446454546400404040784444780047
:100540003844041C0444380048545474545448003B
:100550003C44443C14244400000038043C443C0027
:1005600000007840784478000000784C784C78009F
:1005700000007840404040000000182828287C44B3
:10058000000038447C403C0000005454385454006F
:1005900000007804380478000000444C546444009F
:1005A0000010444C54644400000044487048440027
:1005B00000001C24444444000000446C5454440093
:1005C0000000484878484800000038444444380057
:1005D00000007848484848000000704870404000DB
:1005E000000038404040380000007C10101010001F
:1005F0000000484838087000000038545438100093
:1006000000004428102844000000484848487C0462
:1006100000004848380808000000545454547C0036
:100620000000545454547E02000060203C223C00E0
:1006300000004242724A7200000040407844780054
:10064000000070087808700000004C5272524C0094
:1006500000003C443C44440011241FBECFEFD0E1D5
:10066000DEBFCDBF16E0A0E0B1E0E2EFFEE800E0C3
:100670000BBF02C007900D92A433B107D9F726E053
:10068000A4E3B6E001C01D92A23FB207E1F70E94C9
:100690002B3F0C947747B4CCA89521E0209380069B
:1006A0002091DF063091E0062937310578F120915D
:1006B0009806309199062635310540F5BC012B5F2F
:1006C0003F4F30939906209398061092E0061092BF
:1006D000DF0690913506892F90E0880F991F805092
:1006E00090400E947447809135068F5F8093350655
:1006F000A49A80E185BBA8952FEF81EE94E021506C
:1007000080409040E1F700C0000015BA0895409184
:100710003406E42FF0E0EE0FFF1FE050FF4F608142
:10072000718121E0240F209334066817790720F5A2
:10073000E22FF0E0EE0FFF1FE050FF4F608171816C
:100740008617970760F455E0259F900111242250E9
:1007500031093093990620939806409334062091EE
:10076000A9063091AA068217930730F484E190E03D
:1007700090939906809398068091950690E0209139
:100780009806309199068217930720F49093990662
:10079000809398060895CF93DF9300D000D0CDB713
:1007A000DEB78091630080FD6BC01C821B821A82C1
:1007B0001982BE016F5F7F4FCE0103960E94954262
:1007C0008B819C818531954098F08B819C8188320A
:1007D0009A4070F489819A818431954048F48091DF
:1007E000E6069091E70601969093E7068093E60669
:1007F0008B819C818937954098F08B819C818932CF
:100800009A4070F089819A818431954048F48091B2
:10081000E6069091E70601979093E7068093E60637
:100820008B819C818531954098F08B819C818832A9
:100830009A4070F489819A81853C994048F0809172
:100840009806909199060196909399068093980640
:100850008B819C818937954098F08B819C8189326E
:100860009A4070F089819A81853C994048F0809146
:10087000980690919906019790939906809398060F
:100880000F900F900F900F90DF91CF910895EF92FE
:10089000FF920F931F93CF93DF9300D000D0CDB77B
:1008A000DEB78091340190913501A0913601B0916D
:1008B000370189839A83AB83BC8303E02FEF3FEF3B
:1008C0004CED50E068E470E080E090E0EED72FEF70
:1008D0003FEF4CED50E06FE770E080E090E0E5D74F
:1008E0002FEF3FEF4CED50E066EB70E080E090E0E2
:1008F000DCD72FEF3FEF4CED50E06DEE70E080E085
:1009000090E0D3D72FEF3FEF45EA50E068E470E086
:1009100080E090E00E94CA0C2FEF3FEF45EA50E0E4
:1009200068E470E087E390E00E94CA0C2FEF3FEF8D
:1009300045EA50E068E470E08EE690E00E94CA0C60
:100940002FEF3FEF4EE650E068E470E085EA90E07C
:100950000E94CA0C2FEF3FEF48EA50E068E470E0D5
:100960008CED90E00E94CA0CEE24E394F12C2FE170
:1009700030E04FEF5FEF6AE570E08CE090E048D741
:1009800095E0E92EF12C2FE130E04FEF5FEF61E9C8
:1009900070E08CE090E03CD729E0E22EF12C2FE1D2
:1009A00030E04FEF5FEF68EC70E08CE090E030D724
:1009B00032E0E32EF12C2FE130E04FEF5FEF6AE5FC
:1009C00070E083E490E024D746E0E42EF12C2FE1A0
:1009D00030E04FEF5FEF61E970E083E490E018D71B
:1009E000E12CF12C2FE130E04FEF5FEF68EC70E08D
:1009F00083E490E00DD753E0E52EF12C2FE130E0B9
:100A00004FEF5FEF6AE570E08AE790E001D767E0BB
:100A1000E62EF12C2FE130E04FEF5FEF61E970E05F
:100A20008AE790E0F5D674E0E72EF12C2FE130E074
:100A30004FEF5FEF6AE570E081EB90E0E9D6E8E028
:100A4000EE2EF12C2FE130E04FEF5FEF61E970E027
:100A500081EB90E0DDD6E12CF12C2FE130E04FEF7F
:100A60005FEF68EC70E089E890E0D2D62FE130E0EB
:100A70004FEF5FEF68EC70E083EA90E0C9D6F3E0F7
:100A8000EF2E0FEF1FEF2CE330E04AE550E068E473
:100A900070E081EE90E0F3D7CE0101967C0102E098
:100AA0002FE130E040E058EF64E670E085EF90E041
:100AB00069D6A3E0EA2E0FEF1FEF20E530E04AE50C
:100AC00050E066E970E081EE90E0D9D700EE17E0E3
:100AD0002CED30E04EE051E06EEB70E085EF90E001
:100AE0000E94BC0D20EA30E04CE251E06CED70E079
:100AF0008EE091E00E94BC0D2CED30E04FE051E023
:100B00006EEB70E086EF90E00E94BC0D20EA30E0D2
:100B10004BE251E06CED70E08DE091E00E94BC0D85
:100B20002CED30E040E151E06EEB70E087EF90E0BB
:100B30000E94BC0D20EA30E04AE251E06CED70E02A
:100B40008CE091E00E94BC0D2CED30E041E151E0E1
:100B50006EEB70E088EF90E00E94BC0D20EA30E080
:100B60004AE251E06CED70E08BE091E00E94BC0D38
:100B7000B2E0EB2E0FEF1FEF2CE330E040EA50E045
:100B800063E070E080E590E07AD70F900F900F90CF
:100B90000F90DF91CF911F910F91FF90EF900895EB
:100BA000EF920F931F9383E0E82E0FEF1FEF22E3E6
:100BB00030E040EA50E064E670E084E190E05FD726
:100BC00020E530E04AE550E066E970E081EE90E033
:100BD00056D700EE17E02CED30E04EE051E06EEB22
:100BE00070E085EF90E0C8D720EA30E04CE251E0B9
:100BF0006CED70E08EE091E0BFD72CED30E04FE07F
:100C000051E06EEB70E086EF90E0B6D720EA30E07E
:100C10004BE251E06CED70E08DE091E0ADD72CED52
:100C200030E040E151E06EEB70E087EF90E0A4D758
:100C300020EA30E04AE251E06CED70E08CE091E0B7
:100C40009BD72CED30E041E151E06EEB70E088EF96
:100C500090E092D720EA30E04AE251E06CED70E09B
:100C60008BE091E089D71F910F91EF900895EF925B
:100C7000FF920F931F93CF93DF9300D000D0CDB797
:100C8000DEB77C018091630080FD22C11C821B8243
:100C90001A821982BE016F5F7F4FCE0103960E94B8
:100CA00095420FE110E02DE230E042E550E06AE0CD
:100CB00070E08BE990E071D48B819C81893B9B40F3
:100CC00068F089819A81883D9E4040F489819A81AB
:100CD00089349D4018F089E0809325018B819C81A7
:100CE0008F32994090F08B819C81803F9A4068F4CC
:100CF00089819A81883D9E4040F489819A81893416
:100D00009D4018F085E0809325018B819C81853A78
:100D1000964090F08B819C818C3F984068F489814B
:100D20009A81883D9E4040F489819A8189349D4012
:100D300018F081E0809325018B819C81853A964053
:100D400090F08B819C818C3F984068F489819A81D6
:100D500088349D4040F489819A818D389A4018F0FA
:100D600082E0809325018B819C818F32994090F0A5
:100D70008B819C81803F9A4068F489819A81883474
:100D80009D4040F489819A818D389A4018F086E020
:100D9000809325018B819C81893B9B4060F08981F8
:100DA0009A8188349D4038F489819A818D389A409F
:100DB00010F0109225018B819C81893B9B4068F04B
:100DC00089819A818E3B9A4040F489819A818F3043
:100DD000964018F08AE0809325018B819C81853AAA
:100DE000964090F08B819C818C3F984068F489817B
:100DF0009A818C389A4040F489819A81813D97404C
:100E000018F083E0809325018B819C81853A964080
:100E100090F08B819C818C3F984068F489819A8105
:100E2000803D974040F489819A818D3D954018F02E
:100E300084E0809325018B819C818F32994090F0D2
:100E40008B819C81803F9A4068F489819A818C389B
:100E50009A4040F489819A81813D974018F087E05B
:100E6000809325018B819C818F32994090F08B81FA
:100E70009C81803F9A4068F489819A81803D9740A7
:100E800040F489819A818D3D954018F088E08093E7
:100E900025018B819C818D3D954068F08B819C81E3
:100EA0008C3F984040F489819A818C3D954018F49C
:100EB0008BE0809325018B819C818F32994040F09B
:100EC00089819A818C3D954018F48CE080932501AE
:100ED000809125018A3088F49091380691110DC0D7
:100EE0008093460690E0909337068093360682E022
:100EF000809338068EE080932501809125018A3009
:100F0000A9F48091460634E6839FC0011124909392
:100F100037068093360622E020933806E816F90655
:100F200010F08EE001C08BE08093250180912501B7
:100F30008A30C0F4909138069230A1F48093440630
:100F40002091460690E04AE0249F800D911D1124D7
:100F5000909337068093360683E0809338068EE0C0
:100F600080932501209125012A3010F580913806C3
:100F70008330F1F420934506309146068091440673
:100F80004AE0849FC001112444E6349F800D911DE6
:100F90001124820F911D909337068093360621E02D
:100FA00020933806E816F90668F48BE08093250153
:100FB000809125018B3049F4109237061092360645
:100FC000109238068EE080932501809125018C30A7
:100FD00019F483E2809325010F900F900F900F90EA
:100FE000DF91CF911F910F91FF90EF900895EF92B5
:100FF000FF920F93E0903606F09037062AE0E21653
:10100000F10450F403E02FE130E04FEF5FEF66E1D1
:1010100070E088EC90E0FCD3E0903606F090370664
:10102000C7010A978A35910550F403E02FE130E0BB
:101030004FEF5FEF66E170E084EB90E0E9D3E09082
:101040003606F0903706C7018456910984389340DC
:1010500050F403E02FE130E04FEF5FEF66E170E026
:101060008BE990E0D5D30F91FF90EF9008950F9307
:101070001F93CF93DF93EC018B01809125018E317B
:1010800018F48FE190E0FED31093370600933606F4
:10109000809125018E3128F4FADBCE01E8DDA7DF4F
:1010A000F7CF8FE190E0EED380913606909137062E
:1010B000DF91CF911F910F9108958EE080932501CC
:1010C0000895EF92FF920F931F93CF93DF93CDB7C5
:1010D000DEB728970FB6F894DEBF0FBECDBF809164
:1010E000630080FD50C018861F821E821D82BE01D3
:1010F0006B5F7F4FCE0107960E9495420FE110E093
:101100002EE230E044E650E062E370E082E390E0FB
:1011100044D28F819885853A964090F08F8198854A
:101120008C389A4068F48D819E8184379E4040F4CB
:101130008D819E81813F9A4018F081E08093250146
:101140008F819885853A964088F08F8198858C3874
:101150009A4060F48D819E818C389A4038F48D815C
:101160009E818939984010F0109225018F819885D1
:101170008F32994040F08D819E818C3D954018F4CE
:101180008CE08093250180912501813011F48093BA
:10119000240180912401813061F580913801909182
:1011A0003901A0913A0189839A83AB83CE010196DC
:1011B0007C0104E02FE130E040EE57E062E370E0B4
:1011C00086E490E0DFD200EE17E02EE230E04DE45E
:1011D00050E067E670E087E190E0DFD10FE110E0DA
:1011E0002EE230E04DE450E067E670E086E690E005
:1011F000D4D180912501811102C0109224018091E7
:10120000240181112FC080913B0190913C01A0915C
:101210003D01B0913E0189839A83AB83BC8300E09A
:1012200018EF2EE230E04DE450E067E670E086E62D
:1012300090E0B3D10FE110E02EE230E04DE450E059
:1012400067E670E087E190E0A8D1CE0101967C01CD
:1012500004E02FE130E040E058EF62E370E087E324
:1012600090E090D2809125018C3019F483E2809334
:10127000250128960FB6F894DEBF0FBECDBFDF91D3
:10128000CF911F910F91FF90EF900895CF93C82FAA
:10129000809125018E3118F48FE190E0F3D2C09354
:1012A0002401809125018E3120F4A89579DC09DF95
:1012B000F8CF8FE190E0E6D280912401CF9108959C
:1012C000E2E6F0E090819E7F90839081946090832D
:1012D0009081977F9083A8988BBB8DE08A95F1F7DA
:1012E0000000A89A8081886080830895E2E6F0E09B
:1012F0009081916090839081946090839081977F9A
:101300009083A8988BBB8DE08A95F1F70000A89A8E
:101310008081886080830895CF93C82F892FE6DF6E
:101320008C2FCF91E3CFE2E6F0E020812160208393
:101330002081246020832081277F2083A8988BBB75
:1013400092BB8DE08A95F1F70000A89A80818860B1
:1013500080830895CF93C82F86E3B2DFC13049F070
:1013600030F0C23041F0C33059F488EE07C088E451
:1013700003C088E203C088E8B9DF04C0B7DF0BC050
:10138000CD7F49F48FEE90E090933C0680933B062E
:101390008FE391E008C08FE391E090933C06809347
:1013A0003B068FEE90E090933A0680933906CF91FA
:1013B0000895CF93C82F8FEF8ABB81BB80936100C4
:1013C00081E084BBE2E6F0E080818260808381E09E
:1013D00077DF2FEF89E698E1215080409040E1F7D8
:1013E00000C0000080EC6CDF85E280DF81EC68DF0C
:1013F00081E17CDF85EC64DF8BE278DF8BE276DFF6
:1014000087EC5EDF86E872DF8C2FA4DF8AE358DF8B
:1014100085E06CDF81EB54DF80E068DF88E166DF28
:1014200086EB4EDF8AE062DF82E860DF87E25EDF24
:1014300081E146DF2FEF8DEE92E021508040904019
:10144000E1F700C0000089E2CF913ACF0F931F93DC
:10145000CF93DF938C01EB018AE232DFC8015CDFBE
:10146000CE01DF91CF911F910F9156CF0F931F9314
:10147000CF93DF938C01EB018BE222DFC8014CDFBD
:10148000CE01DF91CF911F910F9146CFCF93DF9384
:10149000EB01BC01DBDFBE01CE01E8DF8CE2DF91B6
:1014A000CF910ECFCF93DF93EA01F0DFCE01DF9132
:1014B000CF9139CF8F929F92AF92BF92CF92DF920E
:1014C000EF92FF920F931F93CF93DF93A895681726
:1014D000790738F48627972768277927862797275B
:1014E000A8952417350738F4422753272427352792
:1014F00042275327A895A0913B06B0913C06FC01DA
:10150000A817B90708F4FD016B01A617B70708F47F
:101510006D018091390690913A06EA01841795078A
:1015200008F4EC0179018217930708F47C01A8956F
:1015300096012F5F3F4F2E1B3F0BD7011196AC1B1F
:10154000BD0B0E943F444B015C01B601CF017EDF21
:10155000A895B701CE018ADF8CE2B2DEA895C12C36
:10156000D12C7601C814D904EA04FB0449F0C8015F
:10157000DADEA8958FEFC81AD80AE80AF80AF2CF7F
:10158000DF91CF911F910F91FF90EF90DF90CF905F
:10159000BF90AF909F908F9008950F931F93411528
:1015A000510579F02115310561F0FA01AB01615067
:1015B0007109260F371FBC01615071096E0F7F1F23
:1015C00079DF1F910F9108952F923F924F925F9272
:1015D0006F927F928F929F92AF92BF92CF92DF9243
:1015E000EF92FF920F931F93CF93DF93CDB7DEB7A8
:1015F00067970FB6F894DEBF0FBECDBF5C01798B45
:10160000688B598748873B872A870F83F12C28E00E
:10161000029FC00111241A821982E8E0F0E0FF8BDA
:10162000EE8B47019C01285F31093B8B2A8BFC0123
:10163000E052F340FD8BEC8BC888D98889819A8170
:10164000C80ED91E8A899B89EE89FF898E1B9F0B44
:101650009C0120583E4F3F872E878C899D898E1B89
:101660009F0BFC01E058FE4FFD87EC871E821D8218
:101670001C821B8287E0682E712C412C512C212C5E
:10168000312CFF81F7FD1EC0EE85FF85849190E02F
:10169000062C02C0959587950A94E2F780FF08C052
:1016A000088519859701A701B6018D819E8107C024
:1016B0000A851B859701A701B6018B819C818A0D44
:1016C0009B1D20C0FF81F03CF0F0EC85FD858491EE
:1016D00090E0062C02C0959587950A94E2F780FF6A
:1016E00009C0088519859701A701B601C501820DBA
:1016F000931D08C00A851B859701A701B601C50186
:10170000840D951D4ADF280C391C480C591CF1E04A
:101710006F1A71082B813C81280D391D3C832B8366
:101720008D819E81880D991D9E838D839FEF691603
:10173000790609F0A6CFEE89FF893197FF8BEE8BF2
:1017400029813A812E0D3F1D3A832983EF2B09F021
:1017500073CF67960FB6F894DEBF0FBECDBFDF9193
:10176000CF911F910F91FF90EF90DF90CF90BF909E
:10177000AF909F908F907F906F905F904F903F9031
:101780002F9008954F925F926F927F928F929F92C7
:10179000AF92BF92CF92DF92EF92FF920F931F937F
:1017A000CF93DF93EC016B014A013901102F88E0E0
:1017B000089F500111242701F20101912F010023FC
:1017C000B1F020913B0630913C06CE0108962817D7
:1017D000390720F4CA0CDB1CC1E0D0E0E12E9301F4
:1017E000A401B601CE01F0DECA0DDB1DE5CFDF910D
:1017F000CF911F910F91FF90EF90DF90CF90BF900E
:10180000AF909F908F907F906F905F904F900895D2
:101810006F927F928F929F92AF92BF92CF92DF9200
:10182000EF92FF920F93CF93DF9300D000D0CDB70C
:10183000DEB76C015B014A013901C70119821A82C6
:101840001B821C824AE0BE016F5F7F4F0E944E44A4
:10185000CE0101967C019301A401B501C60192DF7E
:101860000F900F900F900F90DF91CF910F91FF90FD
:10187000EF90DF90CF90BF90AF909F908F907F9030
:101880006F9008950F931F932091390630913A0677
:1018900060913B0670913C068C0140E050E080E096
:1018A00090E008DE1F910F9108956F927F928F92C2
:1018B0009F92AF92BF92CF92DF92EF92FF920F93DF
:1018C000CF93DF936C01EB017A0159014C01840E37
:1018D000951EB401BBDDBE01CE01C8DD8CE2F0DC9B
:1018E000612C712C6E147F0431F0C5011CDD8FEF6B
:1018F000681A780AF7CF023008F43EC0B401C60176
:10190000A5DDCE010196BC01B1DD8CE2D9DC612CF4
:10191000712C6E147F0431F0C50105DD8FEF681A5C
:10192000780AF7CF023041F1B401C6018FDDCE0154
:101930000296BC019BDD8CE2C3DC612C712C6E1421
:101940007F0431F0C501EFDC8FEF681A780AF7CF1A
:10195000033091F0B401C60179DDCE010396BC01DC
:1019600085DD8CE2ADDCC0E0D0E0CE15DF0521F0F6
:10197000C501D9DC2196F9CFDF91CF910F91FF906E
:10198000EF90DF90CF90BF90AF909F908F907F901F
:101990006F9008956F927F928F929F92AF92BF92B5
:1019A000CF92DF92EF92FF920F93CF93DF93EC01F0
:1019B0006B017A015901BC0149DD46018E0C9F1C67
:1019C000B401C60153DD8CE27BDC612C712C6E14FA
:1019D0007F0431F0C501A7DC8FEF681A780AF7CFD2
:1019E000023008F43EC0CE010196BC012FDDB401E7
:1019F000C6013CDD8CE264DC612C712C6E147F042A
:101A000031F0C50190DC8FEF681A780AF7CF023009
:101A100041F1CE010296BC0119DDB401C60126DDFB
:101A20008CE24EDC612C712C6E147F0431F0C50108
:101A30007ADC8FEF681A780AF7CF033091F0CE0185
:101A40000396BC0103DDB401C60110DD8CE238DC75
:101A5000C0E0D0E0CE15DF0521F0C50164DC2196A1
:101A6000F9CFDF91CF910F91FF90EF90DF90CF9062
:101A7000BF90AF909F908F907F906F9008956F92DE
:101A80007F928F929F92AF92BF92CF92DF92EF920E
:101A90000F931F93CF93DF936C015B01EA01390130
:101AA00048010E2D940101DFB301615071096A0DE7
:101AB0007B1D9401AE01C601F8DE9401A301B501BE
:101AC000C60168DFCE0101979401A301B5018C0D19
:101AD0009D1D60DFDF91CF911F910F91EF90DF90FF
:101AE000CF90BF90AF909F908F907F906F90089510
:101AF000EF92FF920F931F93CF93DF93EB018A0135
:101B00007901BC01640F751FA1DCBE01CE01AEDC02
:101B10008CE2D6DBC0E0D0E0C017D10721F0C701CE
:101B200002DC2196F9CFDF91CF911F910F91FF90A9
:101B3000EF900895EF92FF920F931F93CF93DF934F
:101B4000EB018A017901BC0181DCBE01600F711FCC
:101B5000CE018CDC8CE2B4DBC0E0D0E0C017D10752
:101B600021F0C701E0DB2196F9CFDF91CF911F91E2
:101B70000F91FF90EF9008952F923F924F925F92B6
:101B80006F927F928F929F92AF92BF92CF92DF928D
:101B9000EF92FF920F931F93CF93DF9300D000D06B
:101BA00000D0CDB7DEB76C017B015A0139012801A5
:101BB000261B370B3A8329838A01081B190B17FF51
:101BC00003C0119501951109CA14DB0420F02224E9
:101BD0002A94322C03C022242394312C89819A81A7
:101BE0009E838D8397FF05C09195819591099E8372
:101BF0008D832D813E813195219531093C832B8345
:101C0000E614F70428F08FEF9FEF9A83898304C0CE
:101C100021E030E03A83298348018D819E81881A32
:101C2000990AA201B701C6013DDCC401880F991FC2
:101C30002B813C818217930764F0CA14DB0499F06E
:101C40002D813E81821A930AC20CD31C08171907F2
:101C500044F3E614F70439F0800E911E89819A81CD
:101C6000E80EF91EDECF26960FB6F894DEBF0FBE43
:101C7000CDBFDF91CF911F910F91FF90EF90DF903B
:101C8000CF90BF90AF909F908F907F906F905F901C
:101C90004F903F902F900895AF92BF92CF92DF92D6
:101CA000EF92FF920F931F93CF93DF937C016B0111
:101CB000EA01590198011CDFB501615071096C0DF1
:101CC0007D1D9801AE01C70113DF9801A501B60182
:101CD000C70130DFCE0101979801A501B6018E0D35
:101CE0009F1DDF91CF911F910F91FF90EF90DF909B
:101CF000CF90BF90AF901ECF2F923F924F925F92A6
:101D00006F927F928F929F92AF92BF92CF92DF920B
:101D1000EF92FF920F931F93CF93DF931C012B0140
:101D2000690150E000271127041B150BC1E0D0E02A
:101D3000C41BD50BCC0FDD1FE12CF12CA6015701E4
:101D4000A40CB51CB5013101601A710AC301AADBEC
:101D5000A601B5014801820C931CC401A3DBA601B6
:101D60005201AE18BF08B501C4019CDBA601B50144
:101D7000C30198DBEC16FD06B4F08FEFE81AF80A01
:101D8000C701880F991F01968C0F9D1F22273327AB
:101D9000201B310BE216F30639F40C171D074CF02B
:101DA000C0E0D0E001C0CE010C171D0714F0EC011B
:101DB000C5CF0F5F1F4F9801220F331F2F5F3F4F7B
:101DC000820F931F1016110694F7DF91CF911F9188
:101DD0000F91FF90EF90DF90CF90BF90AF909F90CA
:101DE0008F907F906F905F904F903F902F900895CD
:101DF0004F925F926F927F928F929F92AF92BF921B
:101E0000CF92DF92EF92FF920F931F93CF93DF93C6
:101E1000EC015B014A01390128018601ADDE970121
:101E2000A201B301C401A8DE9501AE01B701C20150
:101E3000A3DEDF91CF911F910F91FF90EF90DF9084
:101E4000CF90BF90AF909F908F907F906F905F905A
:101E50004F900895CF93C82F8A3011F48DE0FADFA8
:101E60005D9BFECFCCB980E090E0CF910895CF92FA
:101E7000DF92EF92FF920F931F93CF93DF93CDB733
:101E8000DEB761970FB6F894DEBF0FBECDBF90E00E
:101E90008A30910508F0EFC1FC01EA5BFF4F0C941A
:101EA0003644A8958AE0EFE3F1E0DE011196019057
:101EB0000D928A95E1F7CE0101967C0101E02FE1B8
:101EC00030E04FEF5FEF63E270E08AE090E05ADCD1
:101ED000A895E091DB068E2F90E08830910508F000
:101EE000CAC1FC01E05BFF4F0C943644B8EAEB2E0C
:101EF000B5E0FB2E04C0A3EAEA2EA5E0FA2E02E02C
:101F00002FE130E04FEF5FEF6EE170E08BEE90E09D
:101F1000B1C1FBE7EF2EF5E0FF2E72C1E1E7EE2E37
:101F2000E5E0FE2E6DC177E6E72E75E0F72E68C17D
:101F3000A89588E0E9E4F1E0DE01119601900D92A8
:101F40008A95E1F786E0E6EAF1E0DE011C96019071
:101F50000D928A95E1F7CE0101967C0101E02FE117
:101F600030E04FEF5FEF64E170E084E190E00ADC85
:101F7000CE010C967C012FE130E04FEF5FEF68E27D
:101F800070E08EE190E0FEDBA8958091890602C1A9
:101F9000A89587E0E1E5F1E0DE01119601900D9250
:101FA0008A95E1F786E0E6EAF1E0DE011C96019011
:101FB0000D928A95E1F7CE0101967C0101E02FE1B7
:101FC00030E04FEF5FEF64E170E084E190E0DADB56
:101FD000CE010C967C012FE130E04FEF5FEF68E21D
:101FE00070E08EE190E0CEDBA89580919006D2C0A3
:101FF000A89587E0E8E5F1E0DE01119601900D92E9
:102000008A95E1F7CE0101967C0101E02FE130E0F5
:102010004FEF5FEF63E270E089E190E0B3DBA895FA
:102020002FE130E04FEF5FEF6EE170E08EEE90E079
:10203000A9DB40EEC42E47E0D42E51E6E52EF12C6C
:102040000EE110E021E630E04AE050E067E570E0A4
:1020500084E190E0CDDE06E311E021E630E042E2EB
:1020600051E067E570E08CE291E0C2DE60EAE62EC6
:10207000F12C0EE110E020EA30E04AE050E06AEA9C
:1020800070E084E190E0B4DE06E311E020EA30E0A5
:1020900042E251E06AEA70E08CE291E0A9DEEBC036
:1020A000A8958BE0EFE5F1E0DE01119601900D922D
:1020B0008A95E1F7CE0101967C0101E02FE130E045
:1020C0004FEF5FEF63E270E08FE090E05BDBA8959D
:1020D0008091E5065FC0A89586E0EAE6F1E0DE01C2
:1020E0001C9601900D928A95E1F78AE0E0E7F1E015
:1020F000DE01119601900D928A95E1F7CE010C96C2
:102100007C0101E02FE130E04FEF5FEF64E170E030
:1021100089E190E037DBCE0101967C012FE130E0D0
:102120004FEF5FEF63E270E08FE090E02BDBA8956C
:102130008091DA062FC0A89586E0EAE6F1E0DE019C
:10214000119601900D928A95E1F785E0EAE7F1E0BA
:10215000DE011C9601900D928A95E1F7CE01019661
:102160007C0101E02FE130E04FEF5FEF64E170E0D0
:1021700089E190E007DBCE010C967C012FE130E095
:102180004FEF5FEF63E270E08FE190E0FBDAA8953C
:102190008091D706813059F110F539E9E32E35E009
:1021A000F32E2EC0A89588E0E3EEF1E0DE01119653
:1021B00001900D928A95E1F7CE0101967C0101E034
:1021C0002FE130E04FEF5FEF63E270E08FE090E0EF
:1021D000D9DAA89580919706813049F018F08230BD
:1021E00059F049C02FE5E22E25E0F22E09C09FE804
:1021F000E92E95E0F92E04C085E8E82E85E0F82E5A
:1022000001E030C0A8958BE0EFE7F1E0DE01119628
:1022100001900D928A95E1F785E0EAE8F1E0DE01B0
:102220001C9601900D928A95E1F7CE0101967C01F2
:1022300001E02FE130E04FEF5FEF64E170E08AE012
:1022400090E0A0DACE010C967C012FE130E04FEF58
:102250005FEF68E270E08EE190E094DAA895CE013D
:1022600001967C012FE130E04FEF5FEF6EE170E00F
:1022700086EE90E087DA61960FB6F894DEBF0FBE67
:10228000CDBFDF91CF911F910F91FF90EF90DF9025
:10229000CF900895CF93DF9300D000D0CDB7DEB7B5
:1022A0008091630080FD21C01C821B821A821982EA
:1022B000BE016F5F7F4FCE0103960E9495428B81D6
:1022C0009C81853C994088F0A89589819A81843CBD
:1022D000994058F4A89589819A818D3D954028F0C0
:1022E000A89581E080938206A8950F900F900F909B
:1022F0000F90DF91CF910895CF93DF9300D000D05E
:10230000CDB7DEB7A8958091630080FD23C01C8205
:102310001B821A821982BE016F5F7F4FCE01039626
:102320000E9495428B819C81853C994098F08981DF
:102330009A81843C994070F489819A818D3D9540C1
:1023400048F0109282068FE19EE40197F1F700C0F9
:102350000000A8950F900F900F900F90DF91CF91F4
:102360000895CF92DF92EF92FF920F931F93A8955B
:1023700080918206811140C0A8950FE110E02CE405
:1023800030E04EE650E06CE870E089E690E005D978
:1023900020E038EF48E264EB70E080EA90E0ACDCEB
:1023A00020E038EF47E264EB70E080EA90E0A4DCE4
:1023B00020E038EF4BE264EB70E080EA90E09CDCD8
:1023C00020E038EF45E264EB70E080EA90E094DCD6
:1023D00000E018EF23E230E045E050E065EA70E00D
:1023E00086E990E0DAD823E230E045E050E065EAA3
:1023F00070E085EA90E0D1D880918206813009F0C2
:102400003EC0A8950FE110E02CE430E04EE650E02D
:102410006CE870E089E690E0C0D820EE37E048E252
:1024200064EB70E080EA90E067DC20EE37E047E2A2
:1024300064EB70E080EA90E05FDC20EE37E04BE296
:1024400064EB70E080EA90E057DC20EE37E045E294
:1024500064EB70E080EA90E04FDC80EEC82E87E00D
:10246000D82E94EBE92EF12C07EB10E028EC30E0AD
:1024700044E950E060EA70E084E990E0B9DC1F9143
:102480000F91FF90EF90DF90CF900895EF92FF9221
:102490000F931F93CF93DF93CDB7DEB764970FB63B
:1024A000F894DEBF0FBECDBFA8950FEF1FEF21E45C
:1024B00030E04FE550E065E070E085E090E0ECDB77
:1024C000A89521E430E04FE550E06BE470E085E052
:1024D00090E0E2DB2BE430E04FE550E061E970E0B2
:1024E00085E090E0D9DB89E0EFE8F1E0DE011196CC
:1024F00001900D928A95E1F785E0EAE8F1E0DE01CE
:10250000509601900D928A95E1F7CE0101967C01DB
:1025100001E02FE130E04FEF5FEF60E570E082E136
:1025200090E030D9CE0140967C012FE130E04FEFB2
:102530005FEF6AE570E083E290E024D90FEF1FEFD0
:1025400021E430E04FE550E065E070E08CED90E094
:10255000A3DB21E430E04FE550E06BE470E08CED6C
:1025600090E09ADB2BE430E04FE550E061E970E069
:102570008CED90E091DB86E0E8E9F1E0DE011A966F
:1025800001900D928A95E1F7CE0101967C0101E060
:102590002FE130E04FEF5FEF60E570E08BEE90E011
:1025A000F1D8CE010A967C012FE130E04FEF5FEFCA
:1025B0006AE570E08CEF90E0E5D88EE4E82E83E0E9
:1025C000F82E2FE130E04FEF5FEF66EE70E08AE02B
:1025D00090E0D8D8C6DE8091830649DC64960FB6B9
:1025E000F894DEBF0FBECDBFDF91CF911F910F9149
:1025F000FF90EF900895EF92FF920F93CF93DF93A8
:10260000CDB7DEB7C458D1090FB6F894DEBF0FBE00
:10261000CDBF9AE0EFE3F1E0DE01AA59BF4F019090
:102620000D929A95E1F79EE0EEE9F1E0DE015E960B
:1026300001900D929A95E1F79EE0ECEAF1E0DE015F
:10264000509601900D929A95E1F79CE0EAEBF1E04B
:10265000DE01AB5BBF4F01900D929A95E1F79BE0D5
:10266000EFE5F1E0DE01AF5ABF4F01900D929A9570
:10267000E1F796E0EAE6F1E0DE01A158BF4F0190F4
:102680000D929A95E1F79AE0E0E7F1E0DE01A45AB5
:10269000BF4F01900D929A95E1F79DE0E6ECF1E0D5
:1026A000DE019C9601900D929A95E1F79FE0E3ED93
:1026B000F1E0DE01119601900D929A95E1F799E013
:1026C000E2EEF1E0DE01A059BF4F01900D929A9524
:1026D000E1F79CE0EBEEF1E0DE01D99601900D927E
:1026E0009A95E1F796E0E7EFF1E0DE01A758BF4FDA
:1026F00001900D929A95E1F7A89590E08A309105A6
:1027000008F06BC0FC01E85AFF4FCE010C94364430
:102710008A599F4F7C0102E02FE130E04FEF5FEFDD
:1027200062E870E030C04E9626C0409624C08B5BB5
:102730009F4F21C08F5A9F4F1EC081589F4F7C01D1
:1027400002E02FE130E04FEF5FEF6EE670E088E2ED
:1027500090E018D8CE01845A9F4F7C012FE130E0E1
:102760004FEF5FEF67E870E08FE090E034C08C9649
:1027700002C080599F4F7C0102E02FE130E04FEF13
:102780005FEF68E770E088E090E025C001967C018B
:1027900002E02FE130E04FEF5FEF68E770E082E0AA
:1027A00090E019C0C9967C0102E02FE130E04FEFC4
:1027B0005FEF6EE670E084E190E00E94C20BCE0114
:1027C00087589F4F7C012FE130E04FEF5FEF67E8C4
:1027D00070E08CE390E00E94C20BCC57DF4F0FB645
:1027E000F894DEBF0FBECDBFDF91CF910F91FF9068
:1027F000EF900895CF92DF92EF92FF920F931F9385
:10280000A89500EE17E021E430E048EC50E06AEAD9
:1028100070E085E090E00E94CD0A0FEF1FEF21E409
:1028200030E048EC50E063E270E085E090E034DABC
:1028300083E7E82E83E0F82E01E02FE130E040EE60
:1028400057E06CE370E088E290E00E94C20B0FEF6B
:102850001FEF20E530E040E550E065E070E08BEEF2
:1028600090E01ADA90EEC92E97E0D92E24E1E22EFC
:10287000F12C03E111E026E430E041E351E066E4AD
:1028800070E085EF90E0B4DA37E1E32EF12C24E438
:1028900030E04FE251E064E470E087EF90E0A8DAC6
:1028A0000FEF1FEF20E530E040E550E064E670E018
:1028B0008BEE90E0F1D945EAE42EF12C03E111E032
:1028C00023E730E041E351E063E770E085EF90E01B
:1028D0008FDA53EAE52EF12C25E730E04FE251E0A4
:1028E00065E770E087EF90E083DA67EBE62E65E05E
:1028F000F62E02E020EE37E040E050E068EC70E0B9
:102900008DE290E00E94C20B1F910F91FF90EF901B
:10291000DF90CF900895CF92DF92EF92FF920F93C6
:102920001F93CF93DF93CDB7DEB765970FB6F894BB
:10293000DEBF0FBECDBFA8958FE0E3EDF1E0DE0175
:10294000119601900D928A95E1F786E0EDEFF1E0A6
:10295000DE01509601900D928A95E1F700EE17E0A6
:1029600021E430E048EC50E06AEA70E085E090E075
:102970000E94CD0A0FEF1FEF21E430E048EC50E059
:1029800063E270E085E090E087D9CE0101967C019A
:1029900001E02FE130E040EE57E06CE370E088E2C8
:1029A00090E00E94C20B0FEF1FEF20E530E040E502
:1029B00050E065E070E08BEE90E06ED980EEC82EBE
:1029C00087E0D82E94E1E92EF12C03E111E026E412
:1029D00030E041E351E066E470E085EF90E008DA32
:1029E00027E1E22EF12C24E430E04FE251E064E4F0
:1029F00070E087EF90E0FCD90FEF1FEF20E530E0AB
:102A000040E550E064E670E08BEE90E045D935EAB1
:102A1000E32EF12C03E111E023E730E041E351E044
:102A200063E770E085EF90E0E3D943EAE42EF12C10
:102A300025E730E04FE251E065E770E087EF90E096
:102A4000D7D9CE0140967C0102E020EE37E040E08D
:102A500050E068EC70E08DE290E00E94C20B659659
:102A60000FB6F894DEBF0FBECDBFDF91CF911F919F
:102A70000F91FF90EF90DF90CF900895CF92DF926B
:102A8000EF92FF920F931F93A89500EE17E021E4B9
:102A900030E048EC50E06AEA70E085E090E00E94A7
:102AA000CD0A0FEF1FEF21E430E048EC50E063E285
:102AB00070E085E090E0F0D88EE4E82E85E0F82E16
:102AC00001E02FE130E040EE57E06CE370E088E297
:102AD00090E00E94C20B0FEF1FEF20E530E040E5D1
:102AE00050E065E070E08BEE90E0D6D890EEC92E15
:102AF00097E0D92E24E1E22EF12C03E111E026E447
:102B000030E041E351E066E470E085EF90E070D999
:102B100037E1E32EF12C24E430E04FE251E064E4AD
:102B200070E087EF90E064D90FEF1FEF20E530E011
:102B300040E550E064E670E08BEE90E0ADD845EA09
:102B4000E42EF12C03E111E023E730E041E351E012
:102B500063E770E085EF90E04BD953EAE52EF12C66
:102B600025E730E04FE251E065E770E087EF90E065
:102B70003FD968ECE62E65E0F62E02E020EE37E065
:102B800040E050E068EC70E08DE290E00E94C20B03
:102B90001F910F91FF90EF90DF90CF900895CF930A
:102BA000DF9300D000D0CDB7DEB78091630080FD09
:102BB00057C01C821B821A821982BE016F5F7F4F31
:102BC000CE0103960E9495428B819C818431954071
:102BD00068F489819A81843A964040F489819A8187
:102BE0008D32914018F082E08093A5068B819C8104
:102BF0008937954090F08B819C81843C994068F4A2
:102C000089819A81843A964040F489819A818D32F3
:102C1000914018F083E08093A5068B819C818932D6
:102C20009A4068F089819A8184379E4040F4898176
:102C30009A81813D974018F081E08093A5068B81B1
:102C40009C81863F994060F48B819C8181349640C1
:102C500038F089819A81813D974010F01092A50645
:102C60008091A5060F900F900F900F90DF91CF915C
:102C70000895CF92DF92EF92FF920F931F93CF931D
:102C8000DF9300D000D000D0CDB7DEB7A89586E0A6
:102C9000EDEFF1E0DE01119601900D928A95E1F7DA
:102CA00000EE17E021E430E048EC50E06AEA70E022
:102CB00085E090E00E94CD0A0FEF1FEF21E430E0A5
:102CC00048EC50E063E270E085E090E00E944C0E3A
:102CD00020E530E040E550E065E070E08BEE90E00C
:102CE0000E944C0EF0EECF2EF7E0DF2EA4E1EA2E8C
:102CF000F12C03E111E026E430E041E351E066E429
:102D000070E085EF90E074D8B7E1EB2EF12C24E46D
:102D100030E04FE251E064E470E087EF90E068D883
:102D20000FEF1FEF20E530E040E550E064E670E093
:102D30008BEE90E00E944C0E15EAE12EF12C03E19F
:102D400011E023E730E041E351E063E770E085EF15
:102D500090E04ED883EAE82EF12C25E730E04FE2F0
:102D600051E065E770E087EF90E042D8CE01019630
:102D70007C0102E020EE37E040E050E068EC70E0DB
:102D80008CE390E00E94C20B80918306811148C0C1
:102D9000E091DB068E2F90E08830910508F040C06E
:102DA000FC01EE59FF4F0C943644E8EAEE2EE5E0C4
:102DB000FE2E04C073EAE72E75E0F72E02E02FE145
:102DC00030E04FEF5FEF65E070E086E490E026C012
:102DD00069E9E62E65E0F62E18C05FE8E52E55E0BD
:102DE000F52E13C045E8E42E45E0F42E0EC03BE777
:102DF000E32E35E0F32E09C021E7E22E25E0F22E86
:102E000004C097E6E92E95E0F92E02E02FE130E0CC
:102E10004FEF5FEF65E070E08EE190E00E94C20B43
:102E200080918306813001F580918906813069F0B7
:102E300038F08230C9F415E8E12E15E0F12E09C012
:102E400089E9E82E85E0F82E04C00FE8E02E05E0C1
:102E5000F02E02E02FE130E04FEF5FEF65E070E031
:102E60008EE190E00E94C20B80918306823001F5D2
:102E700080919006813069F038F08230C9F4F5E82D
:102E8000EF2EF5E0FF2E09C0B9E9EB2EB5E0FB2EE1
:102E900004C0AFE8EA2EA5E0FA2E02E02FE130E010
:102EA0004FEF5FEF65E070E08EE190E00E94C20BB3
:102EB00080918306843001F58091E506813069F0C8
:102EC00038F08230C9F465E8E62E65E0F62E09C0D8
:102ED000E9E9EE2EE5E0FE2E04C07FE8E72E75E07E
:102EE000F72E02E02FE130E04FEF5FEF65E070E09A
:102EF0008EE190E00E94C20B80918306853001F53F
:102F00008091DA06813069F038F08230C9F435E812
:102F1000E32E35E0F32E09C059E9E52E55E0F52EF4
:102F200004C04FE8E42E45E0F42E02E02FE130E04B
:102F30004FEF5FEF65E070E08EE190E00E94C20B22
:102F400080918306863001F58091D706813069F043
:102F500038F08230C9F485E8E82E85E0F82E09C003
:102F600029E9E22E25E0F22E04C09FE8E92E95E043
:102F7000F92E02E02FE130E04FEF5FEF65E070E007
:102F80008EE190E00E94C20B26960FB6F894DEBF49
:102F90000FBECDBFDF91CF911F910F91FF90EF90AA
:102FA000DF90CF900895EF92FF920F931F9380913F
:102FB0007B0690917C060A97A8F4809152068111B5
:102FC0000CC00FE110E02CE330E044E650E06BE48D
:102FD00070E08EE690E00E94CD0A81E08093520678
:102FE0001092840680917B0690917C060A978A3520
:102FF0009105A8F48091840681110CC00FE110E0C6
:103000002CE330E044E650E06BE470E08EE690E0C4
:103010000E94CD0A81E0809384061092520680912E
:103020007B0690917C0684369105E8F081329340CE
:1030300030F087EE93E090937C0680937B0680913E
:103040008406813061F40FE110E02CE330E044E6C7
:1030500050E06BE470E08EE690E00E94CD0A1092A2
:1030600084061092520680918206813079F4E090B5
:103070007B06F0907C0603E02FE130E04FEF5FEF3E
:1030800064E670E082E890E00E94080C809182067D
:1030900081110FC0E0907B06F0907C0603E02FE1E9
:1030A00030E040E058EF64E670E082E890E00E9493
:1030B000080C1F910F91FF90EF900895EF92FF92EF
:1030C0000F931F938091A9069091AA060A97A8F4DE
:1030D00080917A06811111C00FE110E028E230E002
:1030E00048E550E06FEA70E088E090E00E94CD0A89
:1030F00081E080937A061092D8068091A90690917B
:10310000AA0684369105D8F480917B0690917C06BE
:103110000A97A8F08091D806811111C00FE110E044
:1031200028E230E048E550E06FEA70E088E090E0A7
:103130000E94CD0A81E08093D80610927A06809191
:10314000A9069091AA0684369105E8F08132934051
:1031500030F087EE93E09093AA068093A9068091C1
:10316000D806813061F40FE110E028E230E048E554
:1031700050E06FEA70E088E090E00E94CD0A109283
:10318000D80610927A06E090A906F090AA0602E00E
:103190002FE130E04FEF5FEF6EEB70E08EE190E0FB
:1031A0000E94080C1F910F91FF90EF900895EF92ED
:1031B000FF920F931F93809198068A30A8F4809114
:1031C000810681110CC00FE110E024E230E04AE5F5
:1031D00050E064E670E088E090E00E94CD0A81E073
:1031E0008093810610929406809198068A508A35C1
:1031F000A8F48091940681110CC00FE110E024E244
:1032000030E04AE550E064E670E088E090E00E943B
:10321000CD0A81E0809394061092810680919806F1
:103220008436A1F480919406813061F40FE110E0BE
:1032300024E230E04AE550E064E670E088E090E0A7
:103240000E94CD0A109281061092940680919806F1
:10325000843618F084E680939806E0909806F12C66
:1032600002E02FE130E04FEF5FEF6EE670E084E1C7
:1032700090E00E94080C8091E6068A30A8F48091C4
:10328000E106811111C00FE110E024E230E04AE5CF
:1032900050E064E670E08FED90E00E94CD0A81E09E
:1032A0008093E1061092AB068091E6068A508A353B
:1032B000A8F48091AB06811111C00FE110E024E267
:1032C00030E04AE550E064E670E08FED90E00E9467
:1032D000CD0A81E08093AB061092E1068091E6066C
:1032E000843629F41092E1061092AB0602C08436AF
:1032F00018F084E68093E606E090E606F12C02E002
:103300002FE130E04FEF5FEF6EE670E089EE90E086
:103310000E94080C1F910F91FF90EF9008957F92EB
:103320008F929F92AF92BF92CF92DF92EF92FF92D5
:103330000F931F93CF93DF93EC016B015A01490167
:10334000702EA89580915506909156060A97A8F47C
:103350008091DC06811111C00FE110E02EE130E018
:1033600044E650E065507109CE0144970E94CD0AB1
:1033700081E08093DC0610929E0680915506909124
:1033800056060A978A359105C0F480919E068111F0
:1033900014C00FE110E02EE130E044E650E0B60149
:1033A00065507109CE0144970E94CD0A81E0809357
:1033B0009E061092DC0610927D0680915506909133
:1033C000560684369105C0F080917D06811114C0A7
:1033D0000FE110E02EE130E044E650E0B601655028
:1033E0007109CE0144970E94CD0A81E080937D0649
:1033F00010929E061092DC06E0905506F09056065C
:10340000072D9401A501B601CE010E94080CA895D4
:10341000DF91CF911F910F91FF90EF90DF90CF90B0
:10342000BF90AF909F908F907F900895CF92DF9242
:10343000EF92FF920F931F938FE190E00E94420C56
:10344000A89500EE17E021E430E048EC50E06AEA8D
:1034500070E085E090E00E94CD0A0FEF1FEF21E4BD
:1034600030E048EC50E063E270E085E090E00E94DC
:103470004C0E8EE3E82E83E0F82E01E02FE130E0E1
:1034800040EE57E06CE370E088E290E00E94C20BEF
:103490000FEF1FEF20E530E040E550E065E070E021
:1034A0008BEE90E00E944C0E90EEC92E97E0D92E44
:1034B00024E1E22EF12C03E111E026E430E041E3C7
:1034C00051E066E470E085EF90E00E94F80E37E18D
:1034D000E32EF12C24E430E04FE251E064E470E0AC
:1034E00087EF90E00E94F80E0FEF1FEF20E530E02D
:1034F00040E550E064E670E08BEE90E00E944C0EF8
:1035000045EAE42EF12C03E111E023E730E041E34A
:1035100051E063E770E085EF90E00E94F80E53EA17
:10352000E52EF12C25E730E04FE251E065E770E051
:1035300087EF90E00E94F80E67EBE62E65E0F62E2E
:1035400002E020EE37E040E050E068EC70E08DE211
:1035500090E00E94C20B8FE19EE40197F1F700C05A
:1035600000001F910F91FF90EF90DF90CF90089592
:10357000A8958BED92E00E945147813071F4A49A96
:1035800080E185BBA8952FEF82E597E02150804030
:103590009040E1F700C0000015BAA8950895A895DD
:1035A0008BED92E00E945147813021F5A49A80E191
:1035B00085BB2FEF32E597E0215030409040E1F796
:1035C00000C00000A89515BA2FEF32E597E0215012
:1035D00030409040E1F700C00000A89585BB2FEF78
:1035E00032E587E0215030408040E1F700C0000024
:1035F000A89515BA0895A8958BED92E00E945147C1
:10360000813009F048C0A49A80E185BBA8952FEFCE
:1036100032E597E0215030409040E1F700C00000D3
:10362000A89515BAA8952FEF32E597E021503040C4
:103630009040E1F700C00000A89585BBA8952FEF4A
:1036400032E597E0215030409040E1F700C00000A3
:10365000A89515BAA8952FEF32E597E02150304094
:103660009040E1F700C00000A89585BB2FEF32E540
:1036700087E0215030408040E1F700C00000A8956D
:1036800015BA9FEF22E537E0915020403040E1F736
:1036900000C00000A89508951092E606BC9A80919B
:1036A000E606880F81BF10929806139A80919806BB
:1036B000880F809386009FDF8DE490E09093DE0674
:1036C0008093DD060895A8951092990610928D06B4
:1036D000109250061092AE0610928A061092800642
:1036E00010929A06109293061092A8061092510614
:1036F000A8958CED92E00E94594790938F06809395
:103700008E06A8958091830681112AC0A895E09124
:10371000DB068E2F90E08830910510F5FC01E6590C
:10372000FF4F4EE150E00C9436446CEB72E014C055
:103730006EE972E011C060E872E00EC062E672E00D
:103740000BC064E472E008C066E272E005C068E0A5
:1037500072E002C06AEE71E08BE596E00E9441479C
:10376000A895809183068130D1F4A895809189062F
:10377000813069F038F0823091F44EE150E060E938
:1037800071E009C04EE150E06CEC71E004C04EE124
:1037900050E06EEA71E08BE596E00E944147A89503
:1037A000809183068230D1F4A89580919006813073
:1037B00069F038F0823091F44EE150E066E371E058
:1037C00009C04EE150E062E771E004C04EE150E014
:1037D00064E571E08BE596E00E944147A8958091F1
:1037E00083068430C9F48091E506813069F038F0B1
:1037F000823091F44EE150E06CED70E009C04EE192
:1038000050E068E171E004C04EE150E06AEF70E022
:103810008BE596E00E944147A8958091830685300C
:10382000C9F48091DA06813069F038F0823091F481
:103830004EE150E062E870E009C04EE150E06EEB0E
:1038400070E004C04EE150E060EA70E08BE596E085
:103850000E944147A895809183068630C9F48091E3
:10386000D706813069F038F0823091F44EE150E0B3
:1038700068E270E009C04EE150E064E670E004C028
:103880004EE150E066E470E08BE596E00E9441472F
:10389000A89587EC90E00197F1F700C000008091B7
:1038A0005B0690915C0690934D0680934C06809148
:1038B0005D0690915E0690939D0680939C06809194
:1038C0005F068093E306809161068093880680916D
:1038D00063068093B0068091650680938706809189
:1038E000670680939606809169068093950680917D
:1038F0006B068093480680916D0690916E069093BA
:10390000D4068093D30680916F068093AF06809192
:103910008306873021F4809171068093830680911D
:103920007306909174069093D2068093D10680918D
:1039300075069091760690935A0680935906809169
:1039400077069091780690937F0680937E06A895DF
:1039500008958091AE06811117C02091870680914D
:103960007B0690917C06821B9109029768F482E3A2
:103970008093E60681E08093AE0680938006809176
:10398000B006811101C0F4DD2091870630E060911E
:10399000E3064091DF065091E006649FC001659FF9
:1039A000900D11246AE070E00E942244620F731FA0
:1039B00070934B0660934A069091E60640914C0640
:1039C00050914D064617570720F450934B064093ED
:1039D0004A0680919606891710F48093E606809136
:1039E0007B0690917C062817390720F04817590765
:1039F00028F155C02091A8062111F8CF841795070A
:103A0000A8F760914A0670914B062091E60686174A
:103A1000970750F42F5F253618F42093E606E6CF7B
:103A200024E62093E60687C0222319F02150209334
:103A3000E6062091E6062223C9F27DC02091E60623
:103A4000222319F021502093E606841B950B06973C
:103A500068F08091E6068A3010F41092E6068091B4
:103A6000E6068A3018F08A508093E6068091510667
:103A7000811106C094DD81E0809393068093510606
:103A8000209157063091580680918E0690918F06AE
:103A90008217930720F400DE81E0809382068091F4
:103AA0008A0681114FC04091D1065091D206809173
:103AB000870690E08417950708F044C0E0917B06E4
:103AC000F0917C064E175F0729F481E08093A806E9
:103AD00080939A068091A8068130A1F560915306E3
:103AE000709154062091590630915A066217730757
:103AF00078F48091E606E417F50728F48F5F8536A1
:103B000028F084E603C0882319F081508093E606EC
:103B100026173707B8F41092A8068091DF06909117
:103B2000E006821B930B9093E0068093DF0681E012
:103B300080938A0608954817590708F0B0CF20915E
:103B4000E60680CF08958091AE06811117C080915E
:103B5000870690E020917B0630917C0682179307C0
:103B600068F482E38093E60681E08093AE0680935A
:103B700080068091B006811101C0FADCE0918706D1
:103B8000F0E04091E3062091DF063091E006429F8D
:103B9000C001439F900D11246AE070E00E9422440E
:103BA0006E0F7F1F70934B0660934A069091E60656
:103BB00040914C0650914D064617570720F45093FC
:103BC0004B0640934A0680919606891710F480931D
:103BD000E60620917B0630917C06E217F307D0F4CD
:103BE0008091A806811116C02417350798F46091BA
:103BF0004A0670914B068091E6062617370728F48F
:103C00008F5F853628F084E603C0882319F0815041
:103C10008093E6064217530770F58091E6068150BF
:103C20008093E606241B350B2630310558F08A3088
:103C300010F41092E6068091E6068A3018F08A5059
:103C40008093E60680915106811106C0A8DC81E0D0
:103C50008093930680935106209157063091580621
:103C600080918E0690918F068217930720F414DDC1
:103C700081E08093820680918A06811146C040913E
:103C8000D1065091D2068091870690E0841795075F
:103C9000E0F5E0917B06F0917C064E175F0729F472
:103CA00081E08093A80680939A068091A8068130CF
:103CB00061F5609153067091540620915906309138
:103CC0005A066217730778F48091E606E417F50741
:103CD00028F48F5F853628F084E603C0882319F026
:103CE00081508093E6062617370778F41092A806CD
:103CF0008091DF069091E006821B930B9093E00683
:103D00008093DF0681E080938A06089540918806BB
:103D10002091550630915606429FC001439F900D59
:103D200011246AE070E00E9422447093AD06609313
:103D3000AC0680919806853618F084E68093980644
:103D40009091950680919806981710F49093980694
:103D5000809199062091A9063091AA0681110DC083
:103D60002639310520F484E68093980606C026396A
:103D7000310519F081E08093990680919906409170
:103D80009C0650919D068130D9F464177507C0F4E4
:103D9000809198062617370770F48F5F981718F0F0
:103DA0008093980602C09093980680919806853675
:103DB00038F084E603C0882319F081508093980678
:103DC0004617570768F52417350770F48091980651
:103DD0008F5F853608F084E6809398068091980678
:103DE000981710F49093980642175307C8F48091DF
:103DF0009806882319F0815080939806C901841B86
:103E0000950B0B9768F0809198068A3010F4109209
:103E10009806809198068A3018F08A508093980608
:103E2000809196069091E606891710F48093E60635
:103E30004217530740F48091E6068F5F853608F0FD
:103E400084E68093E6060895409188062091550601
:103E500030915606429FC001439F900D11246AE0A5
:103E600070E00E9422447093AD066093AC0680918E
:103E70009806853618F084E680939806909195060A
:103E800080919806981710F490939806809199065F
:103E9000811111C02091A9063091AA062639310559
:103EA00020F484E68093980606C02639310519F07F
:103EB00081E0809399068091990640919C065091EB
:103EC0009D068130F9F464177507E0F42091A90686
:103ED0003091AA06809198062617370770F48F5FF5
:103EE000981718F08093980602C0909398068091D6
:103EF0009806853638F084E603C0882319F081508F
:103F0000809398064617570788F52091A9063091A7
:103F1000AA062417350770F4809198068F5F8536BE
:103F200008F084E68093980680919806981710F41C
:103F30009093980642175307C8F4809198068823F7
:103F400019F0815080939806241B350B2B303105D6
:103F500068F0809198068A3010F41092980680914B
:103F600098068A3018F08A508093980608958091B8
:103F70007B0690917C068B35910510F01092980687
:103F800080919906811113C08091A9069091AA068B
:103F9000883121E0920720F484E68093980607C0D8
:103FA0008831914021F0E4DA81E080939906809194
:103FB0009906813081F48091A9069091AA06813AF0
:103FC000910518F01092980608958837910518F415
:103FD0008AE0809398060895CF93C091B006C130CF
:103FE000D9F480918D06811117C08091870690E0E9
:103FF00020917B0630917C062817390768F0809164
:10400000A9069091AA068A55910990934F0680932C
:104010004E06AEDAC0938D06409188062091550673
:1040200030915606429FC001439F900D11246AE0D3
:1040300070E00E9422447093AD066093AC068091BC
:104040009806853618F084E6809398068091990644
:10405000811112C08091A9069091AA068C3221E0AC
:10406000920720F484E68093980606C08C32914033
:1040700019F081E08093990680919906C0918D0690
:104080008130A1F5C11124C080919C0690919D06BC
:1040900068177907E8F42091A9063091AA06809163
:1040A00098062617370778F48F5F809398069091CB
:1040B0009506981710F49093980680919806853687
:1040C00038F084E603C0882319F081508093980665
:1040D0008091870690E00A9720917B0630917C06BC
:1040E0008217930718F486E480939806C13091F400
:1040F00080914E0690914F060E948703C0939306CD
:104100008091570690915806CD9720F0109258064E
:104110001092570680919C0690919D062091AC06C6
:104120003091AD068217930740F42091B00621111B
:1041300004C08A5591090E948703C0914806C13086
:10414000F9F48091500681111BC080917B069091FB
:104150007C062091D3063091D406821B930B0597E1
:1041600078F42091AF0680914E0690914F06820F11
:10417000911D90934F0680934E06FAD9C093500636
:10418000CF910895BC9A8091E606880F81BF139A5B
:1041900080919806880F8093860080918306811114
:1041A00002C01ADFD6DB80918306813019F41092A9
:1041B0009806C9DC80918306823019F41092E606D5
:1041C0000BDF80918306833011F40E94CB03809132
:1041D0008306843009F49ADD80918306853009F4E2
:1041E00095DD80918306863009F42EDE809183066A
:1041F000873009F4BCDE80918306893069F48091B0
:10420000A9069091AA060E944C03809198068635D3
:1042100018F081E080938206089563EC70E08CEBE7
:1042200092E00E94744762EC71E08EEB92E00E9493
:10423000744766E170E080EC92E00E94744766E1AA
:1042400070E082EC92E00E94744761E070E084ECE0
:1042500092E00E947447A8956EE670E086EC92E0CA
:104260000E94744764E670E088EC92E00E94744714
:1042700064E670E08AEC92E00E94744760E070E0CF
:104280008CEC92E00E947447A89560E070E08EECA0
:1042900092E00E94744760E070E080ED92E00E943E
:1042A000744760E070E082ED92E00E94744760E045
:1042B00070E084ED92E00E94744760E070E086ED6B
:1042C00092E00E94744760E070E088ED92E00E9406
:1042D0007447A89566EE70E08EE992E00E947447FC
:1042E00062EC71E080EA92E00E94744766E170E05F
:1042F00082EA92E00E94744766E170E084EA92E00C
:104300000E94744761E070E086EA92E00E94744780
:10431000A89563E770E088EA92E00E94744764E63B
:1043200070E08AEA92E00E94744764E670E08CEAEA
:1043300092E00E94744760E070E08EEA92E00E9492
:10434000744760E070E080EB92E00E94744760E0A8
:1043500070E082EB92E00E947447A89560E070E004
:1043600084EB92E00E94744760E070E086EB92E09C
:104370000E94744760E070E088EB92E00E9474470E
:1043800060E070E08AEB92E00E947447A89566EEC8
:1043900070E080E892E00E94744762EC71E082E88D
:1043A00092E00E94744766E170E084E892E00E9427
:1043B000744766E170E086E892E00E94744761E02D
:1043C00070E088E892E00E947447A89563E770E087
:1043D0008AE892E00E94744764E670E08CE892E01C
:1043E0000E94744764E670E08EE892E00E94744791
:1043F00060E070E080E992E00E94744760E070E065
:1044000082E992E00E94744760E070E084E992E003
:104410000E947447A89560E070E086E992E00E94EF
:10442000744760E070E088E992E00E94744760E0C1
:1044300070E08AE992E00E94744760E070E08CE9E5
:1044400092E00E947447A89566E970E082E692E0E7
:104450000E94744768EC70E084E692E00E94744722
:1044600066E170E086E692E00E94744766E170E0E3
:1044700088E692E00E94744761E070E08AE692E08C
:104480000E947447A89563E770E08CE692E00E9472
:10449000744764E670E08EE692E00E94744764E63A
:1044A00070E080E792E00E94744760E070E082E78D
:1044B00092E00E94744760E070E084E792E00E941E
:1044C000744760E070E086E792E00E947447A89528
:1044D00060E070E088E792E00E94744760E070E07E
:1044E0008AE792E00E94744760E070E08CE792E017
:1044F0000E94744760E070E08EE792E00E9474478B
:10450000A8956EEB70E084E492E00E94744768EC3A
:1045100070E086E492E00E94744766E170E088E40F
:1045200092E00E94744766E170E08AE492E00E94A3
:10453000744761E070E08CE492E00E947447A895B3
:1045400064E670E08EE492E00E94744764E670E0F6
:1045500080E592E00E94744764E670E082E592E0B4
:104560000E94744760E070E084E592E00E94744726
:1045700060E070E086E592E00E94744760E070E0E1
:1045800088E592E00E947447A89560E070E08AE5B3
:1045900092E00E94744760E070E08CE592E00E9437
:1045A000744760E070E08EE592E00E94744760E03E
:1045B00070E080E692E00E947447A89566EE70E095
:1045C00086E292E00E94744762EC71E088E292E039
:1045D0000E94744766E170E08AE292E00E947447AC
:1045E00066E170E08CE292E00E94744761E070E066
:1045F0008EE292E00E947447A89563E770E080E342
:1046000092E00E94744764E670E082E392E00E94C8
:10461000744764E670E084E392E00E94744760E0CF
:1046200070E086E392E00E94744760E070E088E307
:1046300092E00E94744760E070E08AE392E00E949A
:104640007447A89560E070E08CE392E00E947447A4
:1046500060E070E08EE392E00E94744760E070E0FA
:1046600080E492E00E94744760E070E082E492E0AF
:104670000E947447A89566EE70E088E092E00E9480
:10468000744762EC71E08AE092E00E94744766E150
:1046900070E08CE092E00E94744766E170E08EE08A
:1046A00092E00E94744761E070E080E192E00E9435
:1046B0007447A89563E770E082E192E00E94744736
:1046C00064E670E084E192E00E94744764E670E082
:1046D00086E192E00E94744760E070E088E192E039
:1046E0000E94744760E070E08AE192E00E947447A3
:1046F00060E070E08CE192E00E947447A89560E071
:1047000070E08EE192E00E94744760E070E080E229
:1047100092E00E94744760E070E082E292E00E94C2
:10472000744760E070E084E292E00E947447A895CC
:1047300063EC70E08CEC91E00E94744766E170E0FD
:1047400080ED91E00E94744761E070E084ED91E0BB
:104750000E9474476FE070E086ED91E00E9474471C
:10476000A89564E670E088ED91E00E94744761E0EE
:1047700070E082EE91E00E94744763EC70E084EE9A
:1047800091E00E9474476AE070E086EE91E00E943A
:104790007447A89562EC71E084E791E00E94744749
:1047A00066E170E088E791E00E94744761E070E0A4
:1047B0008AE791E00E9474476EE670E08CE791E032
:1047C0000E947447A89564E670E080E891E00E943A
:1047D000744762E070E088E891E00E94744762EC00
:1047E00071E08AE191E00E94744766E170E08CE13B
:1047F00091E00E94744762E170E08EE191E00E94D6
:104800007447A89564E670E084E291E00E947447E2
:1048100064E670E086E291E00E94744764E070E034
:104820008EE291E00E9474476CE271E084E391E0D3
:104830000E947447A89562EC71E080EC90E00E94C1
:10484000744766E170E082EC90E00E94744766E194
:1048500070E084EC90E00E94744761E070E086ECC8
:1048600090E00E947447A8956EE670E088EC90E0B6
:104870000E94744764E670E08AEC90E00E947447FE
:1048800064E670E08CEC90E00E94744765E070E0B4
:1048900084ED90E00E947447A89562EC71E086E692
:1048A00090E00E94744766E170E08AE690E00E9422
:1048B000744761E070E08CE690E00E9474476EE619
:1048C00070E08EE690E00E947447A89564E670E080
:1048D00082E790E00E94744766E070E08AE790E02B
:1048E0000E94744763EC70E08CEB92E00E94744786
:1048F000A89508956FE070E080EE92E00E94744702
:104900006FE070E08EED92E00E9474476FE070E01F
:104910008CED92E00E94744761E08BED92E00E9482
:10492000674761E08AED92E00C9467478FB9779B07
:10493000FECF8FB10895CF93A39AAB9AAB9880E046
:10494000F5DFC82F80E0F2DFAB9A6C2F70E0762F96
:104950006627682B687F7F7723E0769567952A9591
:10496000E1F780E090E00E94314320E030E040E851
:104970005EE30E9497430E94054370937C06609318
:104980007B06CB01CF910895CF93A79AAF9AAF98AA
:1049900080E0CCDFC82F80E0C9DFAF9A6C2F70E0D9
:1049A000762F6627682B687F7F7723E0769567955B
:1049B0002A95E1F780E090E00E94314320E030E06A
:1049C00040E85EE30E9497430E9405437093AA0665
:1049D0006093A906CB01CF91089586E291E0909370
:1049E000EF068093EE0680917C068F9380917B0684
:1049F0008F9383E092E09F938F930E9471448DE0A8
:104A00008A95F1F70000809156068F9380915506A4
:104A10008F938DE092E09F938F930E9471449DE06D
:104A20009A95F1F70000809198061F928F9387E185
:104A300092E09F938F930E9471448DE08A95F1F7E5
:104A400000008091E6061F928F9382E292E09F938E
:104A50008F930E9471449DE09A95F1F700008CE2DB
:104A600092E09F938F930E9471448DE08A95F1F7B5
:104A700000008091AA068F938091A9068F9384E30A
:104A800092E09F938F930E947144A8958DB79EB733
:104A900046960FB6F8949EBF0FBE8DBF80918206DA
:104AA000811108C08DE392E09F938F930E9471441F
:104AB0000F900F90A89580918206813041F484E494
:104AC00092E09F938F930E9471440F900F909DE00E
:104AD0009A95F1F70000E09183068E2F90E08830E0
:104AE000910508F09DC0FC01EE58FF4F0C94364430
:104AF0008BE492E09F938F930E947144A8950F904E
:104B00000F90E091DB068E2F90E08830910508F041
:104B100087C0FC01E658FF4F0C9436448AE592E0CA
:104B200071C08AE692E06EC082EA92E06BC081EBCF
:104B300092E068C080EC92E065C08FEC92E09F93B9
:104B40008F930E947144A8950F900F9080918906D1
:104B5000813009F452C008F44DC0823009F450C0CD
:104B600008958FED92E09F938F930E947144A895D2
:104B70000F900F9080919006813009F43EC0D0F1E3
:104B8000823009F43DC0089580EF92E042C08EEF7C
:104B900092E09F938F930E947144A8950F900F907D
:104BA0008091E506813049F128F1823049F108957C
:104BB0008FE093E09F938F930E947144A8950F908C
:104BC0000F908091DA068130C1F0A0F08230C1F000
:104BD000089582E293E09F938F930E947144A89579
:104BE0000F900F908091D706813039F018F0823005
:104BF00039F0089585E792E005C084E892E002C0AC
:104C000083E992E09F938F930E94714407C084E3ED
:104C100093E09F938F930E947144A8950F900F90FB
:104C20000895CF92DF92EF92FF920F931F93CF934D
:104C3000DF9300D000D0CDB7DEB7809182068130FF
:104C400009F034C18091910690919206892BD9F494
:104C50000FE110E024E230E04AE550E064E670E065
:104C600088E090E00E94CD0A24E230E04AE550E07E
:104C700064E670E08FED90E00E94CD0AA895A49ABA
:104C8000AC980E944612CC24C394D12C8091820609
:104C9000813009F00BC1A895A0DE8091DD069091CE
:104CA000DE068A35910549F42FEF8DE399E4215012
:104CB00080409040E1F700C00000A89503E02FE19C
:104CC00030E04FEF5FEF69E170E085E890E00E942F
:104CD0008F198091630080FD81C0A8951C821B8282
:104CE0001A821982BE016F5F7F4FCE0103960E9428
:104CF00095428B819C818431954088F489819A8189
:104D0000883D9E4060F489819A81853C994038F0C5
:104D1000D0929206C09291061092A00613D48B8175
:104D20009C818431954098F589819A818C3D95408C
:104D300070F589819A81853F914048F1D092920621
:104D4000C09291061092B10680918306811102C033
:104D50000E94153880918306813011F40E94013B36
:104D600080918306823011F40E94083C8091830672
:104D7000843011F40E940F3D80918306853009F440
:104D8000ADD480918306863011F40E940D37809156
:104D90004706813019F58B819C81853C9940F0F064
:104DA00089819A818C3D9540C8F489819A81853F9B
:104DB0009140A0F0D0929206C09291060E94161ADD
:104DC00080E00E942E410E9499411092920610921A
:104DD00091068FE190E00E94420C23DFACDD0E943F
:104DE000D317A8958FEF91EE24E08150904020409A
:104DF000E1F700C00000C8DDA8950E945E18E090B1
:104E00009806F12C02E02FE130E04FEF5FEF6EE605
:104E100070E08CE190E00E94080CE090E606F12C36
:104E20002FE130E04FEF5FEF6EE670E080EF90E053
:104E30000E94080C80914706813011F40E942B4299
:104E40000E947C1180918206811120CFA8950E943A
:104E5000631BA8950E94B81AA8950E9446120FE1FC
:104E600010E029E130E04AE550E06EE670E088E0CD
:104E700090E00E94CD0A29E130E04AE550E06EE67C
:104E800070E08FED90E00E94CD0A8091470681305E
:104E900021F40E9426410E9465421092560610920B
:104EA00055061092920610929106F0CE0F900F9038
:104EB0000F900F90DF91CF911F910F91FF90EF9086
:104EC000DF90CF900895EF92FF920F931F93CF93AF
:104ED000DF9380919F06813009F047C18FE190E018
:104EE0000E94420C0E948B1485E08093A506C5E0C9
:104EF00080919F06813009F038C10E94CF158091C2
:104F0000A5068230D9F48091D0068F5F8093D006B9
:104F10000FE110E02CE330E046EE50E069E670E08F
:104F200081E090E00E94CD0A22E330E043EC50E0C3
:104F300068E270E088E090E00E94CD0A8091A506CA
:104F40008330D9F48091D00681508093D0060FE150
:104F500010E02CE330E046EE50E069E670E081E0DE
:104F600090E00E94CD0A22E330E043EC50E068E29A
:104F700070E088E090E00E94CD0A8091D0068530F4
:104F800010F01092D0068091D006823081F1B8F4F2
:104F90008823D9F0813009F0C1C077E0E72E76E0B0
:104FA000F72E01E02FE130E04FEF5FEF6CE370E0B0
:104FB00088E090E00E94C20B8EED92E029C0833021
:104FC000B1F1843009F471C0A9C0E0E2EE2EE6E050
:104FD000FE2E01E02FE130E04FEF5FEF6CE370E079
:104FE0008FE090E00E94C20B80EE92E011C06BEF68
:104FF000E62E65E0F62E01E02FE130E04FEF5FEFA7
:105000006CE370E082E390E00E94C20B8CED92E0D2
:105010000E9459477C0103E02FE130E04FEF5FEF42
:1050200062E870E080E590E00E94080C77C043EEF3
:10503000E42E45E0F42E01E02FE130E04FEF5FEF8A
:105040006CE370E088E290E00E94C20B51EFE52E25
:1050500055E0F52E02E02FE130E04FEF5FEF62E820
:1050600070E088E290E00E94C20B8091A506811159
:1050700019C0D3D83FDC3DEAE32E35E0F32E2FE113
:1050800030E04FEF5FEF62E870E088E290E00E946E
:10509000C20B2FEF89E698E1215080409040E1F764
:1050A00000C00000C093A50639C022EDE22E25E025
:1050B000F22E01E02FE130E04FEF5FEF6CE370E0A4
:1050C0008EE190E00E94C20B8BED92E00E9451476E
:1050D000813079F494ECE92E95E0F92E03E02FE18C
:1050E00030E04FEF5FEF62E870E080E590E00E9413
:1050F000C20B8BED92E00E94514781110FC08FEBE4
:10510000E82E85E0F82E03E02FE130E04FEF5FEF6F
:1051100062E870E080E590E00E94C20BD091A506A5
:10512000D13069F410929F06109292061092910667
:105130008FE190E00E94420CD093820672DD809154
:10514000A506811106C081E080939F061092E206B9
:1051500013D0C093A5062FE785EB91E02150804046
:105160009040E1F700C00000C3CEDF91CF911F91C6
:105170000F91FF90EF900895BF92CF92DF92EF9240
:10518000FF920F931F93CF93DF938091E2068111DB
:10519000CFC185E08093A506C9E1D0E025E0C22E0D
:1051A000D12C35E0B32E8091E2068111C1C18091EE
:1051B000D006813009F46FC038F0823009F4DDC0C8
:1051C000843009F441C1A4C180EE92E00E945947A5
:1051D0007C0103E02FE130E040E058EF62E870E04E
:1051E00080E590E00E94080C80EE92E00E94594712
:1051F0009093A4068093A3060E94CF158091A506E4
:105200008230A9F48091A3069091A4060196909310
:10521000A4068093A3060FE110E02CE330E046EEF5
:1052200050E069E670E081E090E00E94CD0A809154
:10523000A5068330A9F48091A3069091A406019756
:105240009093A4068093A3060FE110E02CE330E0D6
:1052500046EE50E069E670E081E090E00E94CD0A01
:105260008091A3069091A4064A9720F0D093A406BB
:10527000C093A3068091A3069091A4060A9720F4F8
:10528000D093A406C093A3066091A3067091A406D0
:1052900080EE92E066C08EED92E00E9459477C015C
:1052A00003E02FE130E040E058EF62E870E080E595
:1052B00090E00E94080C8EED92E00E945947909376
:1052C0008606809385060E94CF158091A5068230C0
:1052D000A9F48091850690918606019690938606A2
:1052E000809385060FE110E02CE330E046EE50E0BD
:1052F00069E670E081E090E00E94CD0A8091A50609
:105300008330A9F480918506909186060197909349
:105310008606809385060FE110E02CE330E046EE30
:1053200050E069E670E081E090E00E94CD0A809153
:105330008506909186064A9720F0D0938606C09302
:10534000850680918506909186060A9720F4D09371
:105350008606C093850660918506709186068EED5F
:1053600092E00E9474472FE788E391E0215080404B
:105370009040E1F700C00000CBC08CED92E00E94AD
:1053800059477C0103E02FE130E040E058EF62E84C
:1053900070E080E590E00E94080C8CED92E00E94A5
:1053A00059479093A2068093A1060E94CF15809141
:1053B000A5068230A9F48091A1069091A2060196DB
:1053C0009093A2068093A1060FE110E02CE330E059
:1053D00046EE50E069E670E081E090E00E94CD0A80
:1053E0008091A5068330A9F48091A1069091A20630
:1053F00001979093A2068093A1060FE110E02CE3A1
:1054000030E046EE50E069E670E081E090E00E9416
:10541000CD0A8091A1069091A2064F9720F0D092DC
:10542000A206C092A1068091A1069091A2060597BE
:1054300020F4D092A206C092A1066091A1067091BC
:10544000A2068CED92E08DCF8BED92E00E94514749
:10545000809349060E94CF158091A506823089F479
:10546000809149068F5F809349060FE110E02CE39D
:1054700030E046EE50E069E670E081E090E00E94A6
:10548000CD0A8091A506833089F480914906815028
:10549000809349060FE110E02CE330E046EE50E047
:1054A00069E670E081E090E00E94CD0A80914906B3
:1054B000823010F01092490680914906813079F4CB
:1054C00094ECE92E95E0F92E03E02FE130E040E086
:1054D00058EF62E870E080E590E00E94C20B809196
:1054E000490681110FC08FEBE82E85E0F82E03E00E
:1054F0002FE130E040E058EF62E870E080E590E0B6
:105500000E94C20B609149068BED92E00E946747B2
:105510008091A506813049F48093E20680939F062E
:105520008FE190E00E94420CCEDCB092A5063BCE0B
:10553000DF91CF911F910F91FF90EF90DF90CF906F
:10554000BF9008959F92AF92BF92CF92DF92EF9259
:10555000FF920F931F93CF93DF938091A006811149
:10556000B1C08FE190E00E94420C0E94FA1385E0E6
:105570008093A50610929F06C0E089E0E82ED1E056
:1055800097E0D92E26E0C22E35E0F32E44E0B42E6B
:1055900053E0A52E62E0962E8091A006811192C064
:1055A0000E94CF158091A506823069F4CF5F0FE18C
:1055B00010E02CE330E046EE50E069E670E081E078
:1055C00090E00E94CD0A8091A506833069F4C15015
:1055D0000FE110E02CE330E046EE50E069E670E0C9
:1055E00081E090E00E94CD0ACA3008F0C0E08C2F24
:1055F0000E94FB128C2F90E08A309105A0F5FC01EF
:10560000EE57FF4F0C94364410929F06109283067B
:105610002AC010929F06D093830625C010929F0641
:105620009092830620C010929F06A09283061BC012
:1056300010929F06B092830616C010929F06F092B9
:10564000830611C010929F06C09283060CC0109270
:105650009F06D092830607C0D0939F0604C0109285
:105660009F06E09283068091A5068130F9F480912F
:105670009F06813049F4109283061092A0068FE1B4
:1056800090E00E94420C1FDCD093A006109292067C
:10569000109291068091830690E090937206809319
:1056A00071068FE190E00E94420CBBDAF092A506F1
:1056B0002FEF80E792E0215080409040E1F700C05A
:1056C00000006ACFDF91CF911F910F91FF90EF9073
:1056D000DF90CF90BF90AF909F900895EF92FF9290
:1056E0000F931F93CF93DF93A8958091B1068111FB
:1056F000F4C08FE190E00E94420C0E943E15809120
:10570000DA0690E090938C0680938B0685E0809378
:10571000A506C1E0D5E08091B1068111DEC0A89553
:105720000E94CF158091A5068230A9F480918B0646
:1057300090918C06019690938C0680938B060FE1D6
:1057400010E02CE330E046EE50E069E670E081E0E6
:1057500090E00E94CD0A8091A5068330A9F4809143
:105760008B0690918C06019790938C0680938B0604
:105770000FE110E02CE330E046EE50E069E670E027
:1057800081E090E00E94CD0A80918B0690918C067A
:10579000039720F010928C0610928B0680918B0656
:1057A00090918C068130910589F1D0F0029709F033
:1057B00046C085E8E82E85E0F82E02E02FE130E0D3
:1057C0004FEF5FEF6DE770E088E290E00E94C20B60
:1057D00082E08093DA064EE150E062E870E02BC090
:1057E00029E9E22E25E0F22E02E02FE130E04FEF32
:1057F0005FEF6DE770E088E290E00E94C20B1092CC
:10580000DA064EE150E06EEB70E015C09FE8E92E3D
:1058100095E0F92E02E02FE130E04FEF5FEF6DE70A
:1058200070E088E290E00E94C20BC093DA064EE17D
:1058300050E060EA70E08BE596E00E94414780917D
:10584000A50681110FC0A895C093B10610929206CB
:1058500010929106C093A0068FE190E00E94420C46
:10586000A895DFD98091A506813059F5A895809338
:10587000B10610929206109291068093A0068FE1D5
:1058800090E00E94420CA8951092E7068091DA06FB
:10589000813069F038F0823091F44EE150E062E8F6
:1058A00070E009C04EE150E06EEB70E004C04EE1E4
:1058B00050E060EA70E08BE596E00E944147A895D1
:1058C00013D0D093A5062FEF80E792E021508040BF
:1058D0009040E1F700C000001ECFDF91CF911F91F3
:1058E0000F91FF90EF900895EF92FF920F931F9307
:1058F000CF938091E70681110C9407378FE190E0F8
:105900000E94420C0E94391685E08093A506C5E0EE
:105910008091E70681110C9407370E94CF15809182
:10592000A5068230D9F48091D6068F5F8093D60683
:105930000FE110E02CE330E046EE50E069E670E065
:1059400081E090E00E94CD0A22E330E043EC50E099
:1059500068E270E088E090E00E94CD0A8091A506A0
:105960008330D9F48091D60681508093D6060FE11A
:1059700010E02CE330E046EE50E069E670E081E0B4
:1059800090E00E94CD0A22E330E043EC50E068E270
:1059900070E088E090E00E94CD0A8091D6068E30BB
:1059A00010F01092D606E091D6068E2F90E08E3041
:1059B000910510F00C94C235FC01E457FF4F809123
:1059C00083060C943644811137C080915B06909118
:1059D0005C06893E934020F010925C0610925B06B4
:1059E00077E3E72E75E0F72E01E02FE130E04FEF8F
:1059F0005FEF62E370E08FE090E00E94C20BE0E3B3
:105A0000EE2EE5E0FE2E2FE130E04FEF5FEF66E493
:105A100070E08CE390E00E94C20BE0905B06F09097
:105A20005C0603E02FE130E04FEF5FEF62E870E0EB
:105A300080E590E00E94080C80918306813009F097
:105A4000B6C780915B0690915C06893E934020F03A
:105A500010925C0610925B0657E3E52E55E0F52E9A
:105A600001E02FE130E04FEF5FEF62E370E08FE0A5
:105A700090E00E94C20B60E3E62E65E0F62E2FE177
:105A800030E04FEF5FEF66E470E08CE390E00E945F
:105A9000C20BE0905B06F0905C067EC7811137C0B8
:105AA00080915D0690915E06893E934020F01092B1
:105AB0005E0610925D0638E1E32E35E0F32E01E03C
:105AC0002FE130E04FEF5FEF62E370E08FE090E0B6
:105AD0000E94C20B4AE0E42E45E0F42E2FE130E0B4
:105AE0004FEF5FEF66E470E08CE390E00E94C20B42
:105AF000E0905D06F0905E0603E02FE130E04FEFAE
:105B00005FEF62E870E080E590E00E94080C809111
:105B10008306813031F48091D6068F5F8093D6065C
:105B200039C08230B9F580915D0690915E06893E5C
:105B3000934020F010925E0610925D0698E1E92EE7
:105B400095E0F92E01E02FE130E04FEF5FEF62E3E7
:105B500070E08FE090E00E94C20B2AE0E22E25E088
:105B6000F22E2FE130E04FEF5FEF66E470E08CE360
:105B700090E00E94C20BE0905D06F0905E0603E0AC
:105B80002FE130E04FEF5FEF62E870E080E590E0FA
:105B90000E94080C809183068430B9F580915D06DF
:105BA00090915E06893E934020F010925E0610921E
:105BB0005D0608E1E02E05E0F02E01E02FE130E087
:105BC0004FEF5FEF62E370E08FE090E00E94C20B66
:105BD0008AE0E82E85E0F82E2FE130E04FEF5FEF0E
:105BE00066E470E08CE390E00E94C20BE0905D06FA
:105BF000F0905E0603E02FE130E04FEF5FEF62E8E8
:105C000070E080E590E00E94080C8091830685306A
:105C1000B9F580915D0690915E06893E934020F033
:105C200010925E0610925D06B8E1EB2EB5E0FB2EF9
:105C300001E02FE130E04FEF5FEF62E370E08FE0D3
:105C400090E00E94C20B1AE0E12E15E0F12E2FE148
:105C500030E04FEF5FEF66E470E08CE390E00E948D
:105C6000C20BE0905D06F0905E0603E02FE130E0AD
:105C70004FEF5FEF62E870E080E590E00E94080C73
:105C800080918306863009F07DC780915D069091F2
:105C90005E06893E934020F010925E0610925D06EB
:105CA000F8E1EF2EF5E0FF2E01E02FE130E04FEFBD
:105CB0005FEF62E370E08FE090E00E94C20BAAE029
:105CC000EA2EA5E0FA2E2FE130E04FEF5FEF66E419
:105CD00070E08CE390E00E94C20BE0905D06F090D3
:105CE0005E06B2C5811136C080915F069091600654
:105CF0004F9720F01092600610925F0672EFE72E29
:105D000074E0F72E01E02FE130E04FEF5FEF62E348
:105D100070E08FE090E00E94C20BEAEDEE2EE4E02E
:105D2000FE2E2FE130E04FEF5FEF66E470E08FE092
:105D300090E00E94C20BE0905F06F090600603E0E6
:105D40002FE130E04FEF5FEF62E870E080E590E038
:105D50000E94080C80918306813009F028C680914A
:105D60005F06909160064F9720F0109260061092A7
:105D70005F0652EFE52E54E0F52E01E02FE130E012
:105D80004FEF5FEF62E370E08FE090E00E94C20BA4
:105D90006AEDE62E64E0F62E2FE130E04FEF5FEF84
:105DA00066E470E08FE090E00E94C20BE0905F0636
:105DB000F0906006F1C5811136C080916106909126
:105DC00062064F9720F0109262061092610632EC44
:105DD000E32E34E0F32E01E02FE130E04FEF5FEFF0
:105DE00062E370E08FE090E00E94C20B4AEAE42E8A
:105DF00044E0F42E2FE130E04FEF5FEF66E470E017
:105E00008FE090E00E94C20BE0906106F090620685
:105E100003E02FE130E04FEF5FEF62E870E080E5F4
:105E200090E00E94080C80918306813031F48091CB
:105E3000D6068F5F8093D60638C08230B1F5809148
:105E40006106909162064F9720F0109262061092C0
:105E5000610692ECE92E94E0F92E01E02FE130E0AA
:105E60004FEF5FEF62E370E08FE090E00E94C20BC3
:105E70002AEAE22E24E0F22E2FE130E04FEF5FEF2E
:105E800066E470E08FE090E00E94C20BE090610653
:105E9000F090620603E02FE130E04FEF5FEF62E841
:105EA00070E080E590E00E94080C809183068430C9
:105EB000B1F580916106909162064F9720F01092A3
:105EC00062061092610602ECE02E04E0F02E01E082
:105ED0002FE130E04FEF5FEF62E370E08FE090E0A2
:105EE0000E94C20B8AEAE82E84E0F82E2FE130E00F
:105EF0004FEF5FEF66E470E08FE090E00E94C20B2E
:105F0000E0906106F090620603E02FE130E04FEF91
:105F10005FEF62E870E080E590E00E94080C8091FD
:105F200083068530B1F580916106909162064F97A6
:105F300020F01092620610926106B2ECEB2EB4E0F3
:105F4000FB2E01E02FE130E04FEF5FEF62E370E006
:105F50008FE090E00E94C20B1AEAE12E14E0F12ECD
:105F60002FE130E04FEF5FEF66E470E08FE090E00C
:105F70000E94C20BE0906106F090620603E02FE100
:105F800030E04FEF5FEF62E870E080E590E00E9464
:105F9000080C80918306863009F0F4C58091610673
:105FA000909162064F9720F010926206109261065F
:105FB000F2ECEF2EF4E0FF2E01E02FE130E04FEFA6
:105FC0005FEF62E370E08FE090E00E94C20BAAEA0C
:105FD000EA2EA4E0FA2E2FE130E04FEF5FEF66E407
:105FE00070E08FE090E00E94C20BE0906106F090BC
:105FF00062062AC4811145C08091630690916406AF
:10600000039730F081E090E09093640680936306FC
:10601000E2E9EE2EE4E0FE2E01E02FE130E04FEF6A
:106020005FEF6CE370E08FE090E00E94C20B809124
:10603000630690916406019779F474ECE72E75E09D
:10604000F72E03E02FE130E04FEF5FEF62E870E002
:1060500080E590E00E94C20B8091630690916406F7
:10606000892B79F46FEBE62E65E0F62E03E02FE145
:1060700030E04FEF5FEF62E870E080E590E00E9473
:10608000C20B80918306813009F045C08091630680
:1060900090916406039730F081E090E0909364065D
:1060A0008093630652E9E52E54E0F52E01E02FE1DE
:1060B00030E04FEF5FEF6CE370E08FE090E00E9424
:1060C000C20B8091630690916406019779F444ECC9
:1060D000E42E45E0F42E03E02FE130E04FEF5FEFD8
:1060E00062E870E080E590E00E94C20B8091630658
:1060F00090916406892B79F43FEBE32E35E0F32E83
:1061000003E02FE130E04FEF5FEF62E870E080E501
:1061100090E00E94C20B80918306823009F045C056
:106120008091630690916406039730F081E090E0DF
:10613000909364068093630622E9E22E24E0F22E17
:1061400001E02FE130E04FEF5FEF6CE370E08FE0B4
:1061500090E00E94C20B80916306909164060197C3
:1061600079F494ECE92E95E0F92E03E02FE130E08C
:106170004FEF5FEF62E870E080E590E00E94C20BB5
:106180008091630690916406892B79F48FEBE82E59
:1061900085E0F82E03E02FE130E04FEF5FEF62E89B
:1061A00070E080E590E00E94C20B809183069CEF36
:1061B000980F923008F4A5C4863009F0E3C48091AA
:1061C000630690916406039730F081E090E090932D
:1061D00064068093630602E9E02E04E0F02E01E0FD
:1061E0002FE130E04FEF5FEF6CE370E08FE090E085
:1061F0000E94C20B8091630690916406019779F426
:1062000014ECE12E15E0F12E03E02FE130E04FEF2A
:106210005FEF62E870E080E590E00E94C20B809141
:10622000630690916406892B09F0ACC4BFEBEB2E9A
:10623000B5E0FB2E03E02FE130E04FEF5FEF62E8C7
:1062400070E080E590E00E94C20B9CC4811137C0D1
:1062500080916506909166068F35914020F01092EE
:10626000660610926506FAE7EF2EF4E0FF2E01E0D5
:106270002FE130E04FEF5FEF62E370E08FE090E0FE
:106280000E94C20BA2E6EA2EA4E0FA2E2FE130E033
:106290004FEF5FEF66E470E08FE090E00E94C20B8A
:1062A000E0906506F090660603E02FE130E04FEFE6
:1062B0005FEF62E870E080E590E00E94080C80915A
:1062C00083068130B9F580916506909166068F3519
:1062D000914020F010926606109265067AE7E72E4C
:1062E00074E0F72E01E02FE130E04FEF5FEF62E363
:1062F00070E08FE090E00E94C20BE2E6EE2EE4E058
:10630000FE2E2FE130E04FEF5FEF66E470E08FE0AC
:1063100090E00E94C20BE0906506F090660603E0F4
:106320002FE130E04FEF5FEF62E870E080E590E052
:106330000E94080C809183068230B9F58091650631
:10634000909166068F35914020F01092660610926B
:1063500065065AE7E52E54E0F52E01E02FE130E026
:106360004FEF5FEF62E370E08FE090E00E94C20BBE
:1063700062E6E62E64E0F62E2FE130E04FEF5FEFAD
:1063800066E470E08FE090E00E94C20BE09065064A
:10639000F090660603E02FE130E04FEF5FEF62E838
:1063A00070E080E590E00E94080C809183069CEFED
:1063B000980F923008F4A5C3863009F0E3C38091AA
:1063C0006506909166068F35914020F01092660622
:1063D000109265063AE7E32E34E0F32E01E02FE158
:1063E00030E04FEF5FEF62E370E08FE090E00E94FB
:1063F000C20B42E6E42E44E0F42E2FE130E04FEFF2
:106400005FEF66E470E08FE090E00E94C20BE090E6
:106410006506F090660618C2811137C08091670644
:10642000909168068636910520F0109268061092C9
:1064300067069AE4E92E94E0F92E01E02FE130E0BE
:106440004FEF5FEF62E370E08FE090E00E94C20BDD
:1064500022E3E22E24E0F22E2FE130E04FEF5FEF57
:1064600066E470E08FE090E00E94C20BE090670667
:10647000F090680603E02FE130E04FEF5FEF62E855
:1064800070E080E590E00E94080C809183068130E6
:10649000B9F580916706909168068636910520F0DF
:1064A00010926806109267060AE4E02E04E0F02ECF
:1064B00001E02FE130E04FEF5FEF62E370E08FE04B
:1064C00090E00E94C20B82E3E82E84E0F82E2FE1D8
:1064D00030E04FEF5FEF66E470E08FE090E00E9405
:1064E000C20BE0906706F090680603E02FE130E011
:1064F0004FEF5FEF62E870E080E590E00E94080CEB
:1065000080918306823031F48091D6068F5F80932C
:10651000D60639C08430B9F5809167069091680637
:106520008636910520F01092680610926706BAE44C
:10653000EB2EB4E0FB2E01E02FE130E04FEF5FEFF8
:1065400062E370E08FE090E00E94C20B12E3E12E64
:1065500014E0F12E2FE130E04FEF5FEF66E470E0E2
:106560008FE090E00E94C20BE0906706F090680612
:1065700003E02FE130E04FEF5FEF62E870E080E58D
:1065800090E00E94080C809183068530B9F58091D7
:106590006706909168068636910520F0109268068D
:1065A00010926706FAE4EF2EF4E0FF2E01E02FE1EF
:1065B00030E04FEF5FEF62E370E08FE090E00E9429
:1065C000C20BA2E3EA2EA4E0FA2E2FE130E04FEF57
:1065D0005FEF66E470E08FE090E00E94C20BE09015
:1065E0006706F090680603E02FE130E04FEF5FEFC1
:1065F00062E870E080E590E00E94080C80918306DC
:106600007DC2811137C08091690690916A068636F5
:10661000910520F010926A06109269067AE1E72E41
:1066200074E0F72E01E02FE130E04FEF5FEF62E31F
:1066300070E08FE090E00E94C20BE2E0EE2EE4E01A
:10664000FE2E2FE130E04FEF5FEF66E470E08FE069
:1066500090E00E94C20BE0906906F0906A0603E0A9
:106660002FE130E04FEF5FEF62E870E080E590E00F
:106670000E94080C80918306813031F48091D60607
:106680008F5F8093D60639C08230B9F58091690654
:1066900090916A068636910520F010926A06109253
:1066A00069065AE1E52E54E0F52E01E02FE130E0D5
:1066B0004FEF5FEF62E370E08FE090E00E94C20B6B
:1066C00062E0E62E64E0F62E2FE130E04FEF5FEF60
:1066D00066E470E08FE090E00E94C20BE0906906F3
:1066E000F0906A0603E02FE130E04FEF5FEF62E8E1
:1066F00070E080E590E00E94080C80918306843071
:10670000B9F58091690690916A068636910520F068
:1067100010926A06109269063AE1E32E34E0F32EF5
:1067200001E02FE130E04FEF5FEF62E370E08FE0D8
:1067300090E00E94C20B42E0E42E44E0F42E2FE1F0
:1067400030E04FEF5FEF66E470E08FE090E00E9492
:10675000C20BE0906906F0906A0603E02FE130E09A
:106760004FEF5FEF62E870E080E590E00E94080C78
:10677000809183068530B9F58091690690916A060B
:106780008636910520F010926A06109269069AE109
:10679000E92E94E0F92E01E02FE130E04FEF5FEFBA
:1067A00062E370E08FE090E00E94C20B22E0E22EF4
:1067B00024E0F22E2FE130E04FEF5FEF66E470E06F
:1067C0008FE090E00E94C20BE0906906F0906A06AC
:1067D00003E02FE130E04FEF5FEF62E870E080E52B
:1067E00090E00E94080C80918306863009F0CAC1AF
:1067F0008091690690916A068636910520F0109284
:106800006A06109269061AE1E12E14E0F12E01E009
:106810002FE130E04FEF5FEF62E370E08FE090E058
:106820000E94C20B82E0E82E84E0F82E2FE130E0D7
:106830004FEF5FEF66E470E08FE090E00E94C20BE4
:10684000E0906906F0906A0603E02FE130E04FEF38
:106850005FEF62E870E080E590E00E94080C92C172
:10686000811129C080917306909174068D329140F8
:1068700020F01092740610927306B2E8EB2EB3E08B
:10688000FB2E01E02FE130E04FEF5FEF6CE370E0B3
:106890008FE090E00E94C20BE0907306F0907406C7
:1068A00003E02FE130E04FEF5FEF62E870E080E55A
:1068B00090E00E94080C80918306813009F077C037
:1068C00080917306909174068D32914020F0109261
:1068D000740610927306A2E8EA2EA3E0FA2E01E0F5
:1068E0002FE130E04FEF5FEF6CE370E08FE090E07E
:1068F0000E94C20BE0907306F09074064DC08111A7
:1069000029C08091750690917606893E934020F0CB
:106910001092760610927506F8EDEF2EF3E0FF2E3A
:1069200001E02FE130E04FEF5FEF6CE370E08FE0CC
:1069300090E00E94C20BE0907506F090760603E0AE
:106940002FE130E04FEF5FEF62E870E080E590E02C
:106950000E94080C80918306813049F5809175066C
:1069600090917606893E934020F010927606109220
:106970007506E8EDEE2EE3E0FE2E01E02FE130E0BB
:106980004FEF5FEF6CE370E08FE090E00E94C20B8E
:10699000E0907506F090760603E02FE130E04FEFCF
:1069A0005FEF62E870E080E590E00E94080C809163
:1069B0008306823009F4A5C09CEF980F923008F04E
:1069C0009DC09FC0811190C080916B0690916C0614
:1069D000039720F010926C0610926B0670EFE72E72
:1069E00073E0F72E01E02FE130E04FEF5FEF6CE353
:1069F00070E08EE190E00E94C20B80916B06909156
:106A00006C06019779F464ECE62E65E0F62E03E05F
:106A10002FE130E04FEF5FEF62E870E080E590E05B
:106A20000E94C20B80916B0690916C06892B79F4C1
:106A30005FEBE52E55E0F52E03E02FE130E04FEF60
:106A40005FEF62E870E080E590E00E94C20B809109
:106A50006B068093480648C0811146C08091480665
:106A6000811108C08DC081113FC0809148068111FD
:106A70009EC186C0813009F085C080916D069091DD
:106A80006E06893E934020F010926E0610926D06BD
:106A90003AE7E32E34E0F32E01E02FE130E04FEF50
:106AA0005FEF62E370E08FE090E00E94C20B42EC87
:106AB000E42E43E0F42E2FE130E04FEF5FEF66E489
:106AC00070E08FE090E00E94C20BE0906D06F090C5
:106AD0006E0603E02FE130E04FEF5FEF62E870E019
:106AE00080E590E00E94080C80918306813049F097
:106AF000823039F0843029F0853019F0863009F081
:106B000041C08091D6068F5F8093D6063BC0882314
:106B100021F09FEF980F923018F41092D6062BC0F8
:106B2000843049F58091770690917806893E9340AC
:106B300020F010927806109277068BE5E82E83E01D
:106B4000F82E01E02FE130E04FEF5FEF6CE370E0F3
:106B50008FE090E00E94C20BE0907706F0907806FC
:106B600003E02FE130E04FEF5FEF62E870E080E597
:106B700090E00E94080C809183068550823010F4CA
:106B80001092D6068091A506813009F0F3C080935B
:106B9000E7061092B10680918306811128C0E0912A
:106BA0008B06F0918C06E830F10508F5E656FF4FAC
:106BB0004EE150E00C9436446CEB72E014C06EE988
:106BC00072E011C060E872E00EC062E672E00BC0D5
:106BD00064E472E008C066E272E005C068E072E05A
:106BE00002C06AEE71E08BE596E00E945E478091FC
:106BF00083068130E1F480918B0690918C06813080
:106C0000910569F038F0029791F44EE150E060E9A7
:106C100071E009C04EE150E06CEC71E004C04EE15F
:106C200050E06EEA71E08BE596E00E945E4780914D
:106C300083068230E1F480918B0690918C0681303E
:106C4000910569F038F0029791F44EE150E066E367
:106C500071E009C04EE150E062E771E004C04EE12E
:106C600050E064E571E08BE596E00E945E4780911C
:106C700083068430E1F480918B0690918C068130FC
:106C8000910569F038F0029791F44EE150E06CED17
:106C900070E009C04EE150E068E171E004C04EE1EF
:106CA00050E06AEF70E08BE596E00E945E478091CD
:106CB00083068530E1F480918B0690918C068130BB
:106CC000910569F038F0029791F44EE150E062E8E6
:106CD00070E009C04EE150E06EEB70E004C04EE1A0
:106CE00050E060EA70E08BE596E00E945E4780919C
:106CF00083068630E1F480918B0690918C0681307A
:106D0000910569F038F0029791F44EE150E068E2A5
:106D100070E009C04EE150E064E670E004C04EE16E
:106D200050E066E470E08BE596E00E945E478FE1FC
:106D300090E00E94420C80918306811101C075D1C0
:106D400080918306813009F45CD48091830682307F
:106D500009F45ED580918306843009F460D6809171
:106D60008306853011F40E946E2B80918306863055
:106D700009F453D08091A50681110CC081E0809365
:106D8000E7061092B106109279068FE190E00E941A
:106D9000420CEED2C093A5068FE798E321E0815024
:106DA00090402040E1F700C000000C94882C813016
:106DB00009F0E8CE80916F0690917006893E93406D
:106DC00020F01092700610926F069BEAE92E93E075
:106DD000F92E01E02FE130E04FEF5FEF62E370E06A
:106DE0008FE090E00E94C20B28E9E22E23E0F22E11
:106DF0002FE130E04FEF5FEF66E470E08FE090E06E
:106E00000E94C20BE0906F06F090700662CECF91A8
:106E10001F910F91FF90EF900895EF92FF920F93C3
:106E20001F93CF93DF93A8958091B1068111F6C08F
:106E30008FE190E00E94420C0E943E158091D7069F
:106E400090E090938C0680938B0685E08093A50656
:106E5000C1E0D5E08091B1068111E0C0A8950E9403
:106E6000CF158091A5068230A9F480918B06909170
:106E70008C06019690938C0680938B060FE110E0B0
:106E80002CE330E046EE50E069E670E081E090E00F
:106E90000E94CD0A8091A5068330A9F480918B06CB
:106EA00090918C06019790938C0680938B060FE14E
:106EB00010E02CE330E046EE50E069E670E081E05F
:106EC00090E00E94CD0A80918B0690918C060397EA
:106ED00020F010928C0610928B0680918B06909178
:106EE0008C068130910589F1D0F0029709F046C0F7
:106EF00085E8E82E85E0F82E02E02FE130E04FEF44
:106F00005FEF6DE770E088E290E00E94C20B82E0E4
:106F10008093D7064EE150E068E270E02BC029E98B
:106F2000E22E25E0F22E02E02FE130E04FEF5FEF9E
:106F30006DE770E088E290E00E94C20B1092D706E5
:106F40004EE150E064E670E015C09FE8E92E95E060
:106F5000F92E02E02FE130E04FEF5FEF6DE770E0D8
:106F600088E290E00E94C20BC093D7064EE150E049
:106F700066E470E08BE596E00E9441478091A506AB
:106F8000811110C0A895C093B1061092920610927C
:106F90009106C093A0068FE190E00E94420CA89554
:106FA0000E9411268091A506813061F5A8958093F5
:106FB000B10610929206109291068093A0068FE17E
:106FC00090E00E94420CA8951092E7068091D706A7
:106FD000813069F038F0823091F44EE150E068E29F
:106FE00070E009C04EE150E064E670E004C04EE19C
:106FF00050E066E470E08BE596E00E944147A8957A
:107000000E94742CD093A5062FEF80E792E02150C8
:1070100080409040E1F700C000001CCFDF91CF918D
:107020001F910F91FF90EF900895AF92BF92CF9272
:10703000DF92EF92FF920F931F93CF93DF93A89568
:107040008091B106811189C18FE190E00E94420CCC
:107050000E943E158091DB0690E090938C06809311
:107060008B0685E08093A506E7E0DE2EF6E0CF2EC6
:10707000D5E0A4E0BA2EB3E0AB2EC1E08091B1061A
:1070800081116BC1A8950E94CF158091A506823011
:10709000A9F480918B0690918C06019690938C06B2
:1070A00080938B060FE110E02CE330E046EE50E0D9
:1070B00069E670E081E090E00E94CD0A8091A5062B
:1070C0008330A9F480918B0690918C060197909360
:1070D0008C0680938B060FE110E02CE330E046EE47
:1070E00050E069E670E081E090E00E94CD0A809176
:1070F0008B0690918C06089720F010928C061092C7
:107100008B06E0918B06F0918C06E830F10508F0D3
:10711000BEC0EE55FF4F0C94364478EAE72E75E07A
:10712000F72E02E02FE130E04FEF5FEF6DE770E008
:1071300082E390E00E94C20B1092DB064EE150E029
:107140006CEB72E09AC063EAE62E65E0F62E02E090
:107150002FE130E04FEF5FEF6DE770E082E390E00A
:107160000E94C20BC093DB064EE150E06EE972E074
:1071700084C059E9E52E55E0F52E02E02FE130E01C
:107180004FEF5FEF6DE770E088E290E00E94C20B86
:1071900082E08093DB064EE150E060E872E06DC073
:1071A0004FE8E42E45E0F42E02E02FE130E04FEF0F
:1071B0005FEF6DE770E088E290E00E94C20BA09262
:1071C000DB064EE150E062E672E057C035E8E32EA0
:1071D00035E0F32E02E02FE130E04FEF5FEF6DE797
:1071E00070E088E290E00E94C20BB092DB0644E1BE
:1071F00050E064E472E041C02BE7E22E25E0F22E7D
:1072000002E02FE130E04FEF5FEF6DE770E088E2E2
:1072100090E00E94C20BD093DB064EE150E066E2A4
:1072200072E02BC091E7E92E95E0F92E02E02FE104
:1072300030E04FEF5FEF6DE770E088E290E00E9492
:10724000C20BC092DB064EE150E068E072E015C070
:1072500087E6E82E85E0F82E02E02FE130E04FEFE0
:107260005FEF6DE770E088E290E00E94C20BD09281
:10727000DB064EE150E06AEE71E08BE596E00E949D
:1072800041478FE59AEE0197F1F700C00000809129
:10729000A50681110FC0A895C093B1061092920661
:1072A00010929106C093A0068FE190E00E94420CDC
:1072B0000E9411268091A506813009F041C0A89551
:1072C0008093B10610929206109291068093A006C8
:1072D0008FE190E00E94420C1092E706E091DB06FD
:1072E0008E2F90E08830910540F5FC01E655FF4F68
:1072F0004EE150E00C9436446CEB72E014C06EE941
:1073000072E011C060E872E00EC062E672E00BC08D
:1073100064E472E008C066E272E005C068E072E012
:1073200002C06AEE71E08BE596E00E9441478FE56E
:107330009AEE0197F1F700C00000A8950E94742C06
:10734000D093A506A8959FEF20E782E091502040BA
:107350008040E1F700C0000091CEDF91CF911F91F6
:107360000F91FF90EF90DF90CF90BF90AF90089576
:10737000CF93C1E080917906811141C1E091D60699
:107380008E2F90E08E30910508F030C1FC01EE5454
:10739000FF4F0C94364460915B0670915C067093CD
:1073A0004D0660934C068EE591E00E94370890935D
:1073B0004D0680934C0690935C0680935B060DC14E
:1073C00060915D0670915E0670939D0660939C06C9
:1073D00082EC91E00E94370890939D0680939C0672
:1073E00090935E0680935D06F8C060915F06709191
:1073F00060066093E306772789E190E00E943708F2
:107400008093E30699279093600680935F06E5C01A
:10741000609161067091620660938806772789E122
:1074200090E00E943708809388069927909362061F
:1074300080936106D2C0809163068093B0060E945B
:1074400046098093B00690E09093640680936306AB
:10745000C4C06091650670916606609387067727C1
:1074600088EC90E00E9437088093870699279093D4
:10747000660680936506B1C06091670670916806E4
:1074800060939606772784E690E00E943708809301
:107490009606992790936806809367069EC0609130
:1074A000690670916A0660939506772784E690E0F6
:1074B0000E94370880939506992790936A068093D7
:1074C00069068BC060917306709174067093D20642
:1074D0006093D10688EC90E00E9437089093D20622
:1074E0008093D106909374068093730676C0609162
:1074F00075067091760670935A066093590684E675
:1075000090E00E94370890935A0680935906909312
:1075100076068093750661C080916B06809348065D
:107520000E944609823018F48093480602C01092E7
:1075300048068091480690E090936C0680936B0615
:107540004CC080914806811103C01092D6064EC0EF
:10755000813009F04BC060916D0670916E0670939A
:10756000D4066093D3068AEF90E00E943708909388
:10757000D4068093D30690936E0680936D062DC03B
:1075800080914806882309F3813081F560916F0668
:10759000709170066093AF06772786E490E00E94B2
:1075A00037088093AF0699279093700680936F06F3
:1075B00014C0609177067091780670937F0660938F
:1075C0007E0684E893E00E94370890937F068093BC
:1075D0007E0690937806809377062FE788E391E004
:1075E000215080409040E1F700C00000C093790630
:1075F0001092E7060E945D080E94742CBBCECF91CA
:107600000895EF92FF920F931F93CF93DF93A89566
:107610008091B1068111F5C08FE190E00E94420C8B
:107620000E943E158091890690E090938C0680938D
:107630008B0685E08093A506C1E0D5E08091B10678
:107640008111DFC0A8950E94CF158091A5068230D8
:10765000A9F480918B0690918C06019690938C06EC
:1076600080938B060FE110E02CE330E046EE50E013
:1076700069E670E081E090E00E94CD0A8091A50665
:107680008330A9F480918B0690918C06019790939A
:107690008C0680938B060FE110E02CE330E046EE81
:1076A00050E069E670E081E090E00E94CD0A8091B0
:1076B0008B0690918C06039720F010928C06109206
:1076C0008B06A89580918B0690918C068130910550
:1076D00089F1D0F0029709F046C085E8E82E85E0F0
:1076E000F82E02E02FE130E04FEF5FEF6DE770E042
:1076F00088E290E00E94C20B82E0809389064EE10E
:1077000050E060E971E02BC029E9E22E25E0F22E7D
:1077100002E02FE130E04FEF5FEF6DE770E088E2CD
:1077200090E00E94C20B109289064EE150E06CEC92
:1077300071E015C09FE8E92E95E0F92E02E02FE1F7
:1077400030E04FEF5FEF6DE770E088E290E00E947D
:10775000C20BC09389064EE150E06EEA71E08BE502
:1077600096E00E9441478091A50681110FC0A8951F
:10777000C093B1061092920610929106C093A00693
:107780008FE190E00E94420C0E9411268091A50694
:10779000813059F5A8958093B10610929206109207
:1077A00091068093A0068FE190E00E94420C109217
:1077B000E70680918906813069F038F0823091F4D3
:1077C0004EE150E060E971E009C04EE150E06CEC40
:1077D00071E004C04EE150E06EEA71E08BE596E0A6
:1077E0000E944147A8950E94742CD093A5062FEFC4
:1077F00080E792E0215080409040E1F700C0000017
:107800001DCFDF91CF911F910F91FF90EF900895C1
:10781000EF92FF920F931F93CF93DF93A8958091E0
:10782000B1068111F5C08FE190E00E94420C0E94E8
:107830003E158091900690E090938C0680938B0685
:1078400085E08093A506C1E0D5E08091B106811165
:10785000DFC0A8950E94CF158091A5068230A9F4BB
:1078600080918B0690918C06019690938C06809364
:107870008B060FE110E02CE330E046EE50E069E6C5
:1078800070E081E090E00E94CD0A8091A5068330EF
:10789000A9F480918B0690918C06019790938C06A9
:1078A00080938B060FE110E02CE330E046EE50E0D1
:1078B00069E670E081E090E00E94CD0A80918B063D
:1078C00090918C06039720F010928C0610928B06F4
:1078D00080918B0690918C068130910589F1D0F0D2
:1078E000029709F046C085E8E82E85E0F82E02E010
:1078F0002FE130E04FEF5FEF6DE770E088E290E05E
:107900000E94C20B82E0809390064EE150E066E355
:1079100071E02BC029E9E22E25E0F22E02E02FE1F2
:1079200030E04FEF5FEF6DE770E088E290E00E949B
:10793000C20B109290064EE150E062E771E015C074
:107940009FE8E92E95E0F92E02E02FE130E04FEFBD
:107950005FEF6DE770E088E290E00E94C20BC09399
:1079600090064EE150E064E571E08BE596E00E9400
:1079700041478091A506811110C0A895C093B1061A
:107980001092920610929106C093A0068FE190E0AB
:107990000E94420CA8950E9411268091A506813074
:1079A00059F5A8958093B10610929206109291060F
:1079B0008093A0068FE190E00E94420C1092E706AF
:1079C00080919006813069F038F0823091F44EE178
:1079D00050E066E371E009C04EE150E062E771E01B
:1079E00004C04EE150E064E571E08BE596E00E9452
:1079F0004147A8950E94742CD093A5062FEF80E7ED
:107A000092E0215080409040E1F700C000001DCF7F
:107A1000DF91CF911F910F91FF90EF900895EF921A
:107A2000FF920F931F93CF93DF93A8958091B10698
:107A30008111F6C08FE190E00E94420C0E943E1539
:107A40008091E50690E090938C0680938B0685E00C
:107A50008093A506C1E0D5E08091B1068111E0C018
:107A6000A8950E94CF158091A5068230A9F4809137
:107A70008B0690918C06019690938C0680938B06D2
:107A80000FE110E02CE330E046EE50E069E670E0F4
:107A900081E090E00E94CD0A8091A5068330A9F490
:107AA00080918B0690918C06019790938C06809321
:107AB0008B060FE110E02CE330E046EE50E069E683
:107AC00070E081E090E00E94CD0A80918B06909159
:107AD0008C06039720F010928C0610928B068091F2
:107AE0008B0690918C068130910589F1D0F0029738
:107AF00009F046C085E8E82E85E0F82E02E02FE187
:107B000030E04FEF5FEF6DE770E088E290E00E94B9
:107B1000C20B82E08093E5064EE150E06CED70E030
:107B20002BC029E9E22E25E0F22E02E02FE130E021
:107B30004FEF5FEF6DE770E088E290E00E94C20BCC
:107B40001092E5064EE150E068E171E015C09FE853
:107B5000E92E95E0F92E02E02FE130E04FEF5FEFE4
:107B60006DE770E088E290E00E94C20BC093E506EA
:107B70004EE150E06AEF70E08BE596E00E944147ED
:107B80008091A506811110C0A895C093B1061092EE
:107B9000920610929106C093A0068FE190E00E9499
:107BA000420CA8950E9411268091A506813061F5AE
:107BB000A8958093B1061092920610929106809338
:107BC000A0068FE190E00E94420CA8951092E70673
:107BD0008091E506813069F038F0823091F44EE111
:107BE00050E06CED70E009C04EE150E068E171E0FA
:107BF00004C04EE150E06AEF70E08BE596E00E9431
:107C00004147A8950E94742CD093A5062FEF80E7DA
:107C100092E0215080409040E1F700C000001CCF6E
:107C2000DF91CF911F910F91FF90EF9008950F93E7
:107C30001F9380918206811199C08091DD069091F9
:107C4000DE068335910591F581E0809382060E94DE
:107C50004C1B0FE110E02CE330E044E650E06BE415
:107C600070E08EE690E00E94CD0A24E230E04AE522
:107C700050E064E670E088E090E00E94CD0A24E2E3
:107C800030E04AE550E064E670E088E090E00E9471
:107C9000CD0A24E230E04AE550E064E670E08FED82
:107CA00090E00E94CD0A0E941126A8950E94ED2422
:107CB0000E94C220A89503E02FE130E04FEF5FEF74
:107CC00069E170E085E890E00E948F190E949B2492
:107CD0000E944A11809182068130A9F5A8950E94E0
:107CE0004C1B0FE110E02CE330E044E650E06BE485
:107CF00070E08EE690E00E94CD0A24E230E04AE592
:107D000050E064E670E088E090E00E94CD0A24E252
:107D100030E04AE550E064E670E088E090E00E94E0
:107D2000CD0A24E230E04AE550E064E670E08FEDF1
:107D300090E00E94CD0A80914706813009F4D5D1A8
:107D40000E941126A8952FEF81EE94E021508040EB
:107D50009040E1F700C000000E94D3170E94C424A5
:107D60000E945E181F910F910C94D7181F910F91CC
:107D700008951F920F920FB60F9211248F939F9325
:107D80008CB190E09093DE068093DD069F918F91F9
:107D90000F900FBE0F901F9018951F920F920FB665
:107DA0000F9211242F938F939F938091550690915A
:107DB00056060196883E23E0920728F490935606D3
:107DC0008093550604C01092560610925506809175
:107DD0008006811105C01092E0061092DF060BC0EC
:107DE000813049F48091DF069091E00601969093EE
:107DF000E0068093DF0680919A06811105C01092FB
:107E00005406109253060BC0813049F480915306FA
:107E10009091540601969093540680935306809156
:107E20009306811105C010925806109257060BC098
:107E3000813049F4809157069091580601969093AD
:107E40005806809357069F918F912F910F900FBEE8
:107E50000F901F9018958091640088608093640053
:107E6000809165008860809365002FEF89E698E136
:107E7000215080409040E1F700C000008FEF8ABBA6
:107E800081BB80936100C1E0C4BBA89588EA8FBD27
:107E90008CE08EBD1DBC1CBC17BC16BC8AE78BBD1C
:107EA00082E18ABD19BC18BC10927900109278004A
:107EB00080E187BF10BE87E683BF12BE11BE81E896
:107EC00080938B0085E080938A0010928900109245
:107ED000880010928100109280001092870010920A
:107EE00086001092850010928400109283001092F8
:107EF00082001BB888E98AB986E0809395001092C9
:107F000090008FE289B98FE181BD8FE081BDA89596
:107F1000F9D2A89581E00E94D909A8958FE190E057
:107F20000E94420CA895C09382061092830610927C
:107F3000560610925506109298061092520610920C
:107F400081061092E10610927A0680E590E0909307
:107F5000DE068093DD06809164008E7F809364004E
:107F600080916500816080936500C0934706A29A66
:107F7000AA9A809164008260809364008091650079
:107F80008260809365007894A49AAC9A2FEF85EA7A
:107F90009EE0215080409040E1F700C00000A8958D
:107FA000AC988AED92E07DD7813011F4A8950FC08E
:107FB0000E940D21A8950E947A24A89561E08BED7E
:107FC00092E085D7A89561E08AED92E080D7A895E8
:107FD00080918206813021F4A8950E941126A895EF
:107FE000A89525DEF4CF80916400806180936400C1
:107FF0008091650080618093650080916400886055
:108000008093640080916500877F809365008091F4
:108010003F06909140068536910500F580916400F9
:108020008460809364008091650084608093650023
:1080300087EB9BE00197F1F700C00000A8958091C5
:1080400065008B7F8093650080913F06909140068C
:1080500001969093400680933F06D9CF80916500AA
:1080600088608093650008958091640080618093AA
:108070006400809165008F7E80936500809164002C
:1080800088608093640080916500877F809365009D
:1080900080913F06909140068536910500F58091CC
:1080A00064008460809364008091650084608093A4
:1080B000650087EB9BE00197F1F700C00000A895F1
:1080C000809165008B7F8093650080913F06909141
:1080D000400601969093400680933F06D9CF809149
:1080E0006500886080936500089582EE92E0D9D69D
:1080F0008093E906A8958091640080618093640074
:108100008091650080618093650080916400886043
:108110008093640080916500877F809365008091E3
:10812000E90624E6829FC001112420913D0630918A
:108130003E062817390700F580916400846080931B
:1081400064008091650084608093650087EB9BE00C
:108150000197F1F700C00000A895809165008B7F22
:108160008093650080913D0690913E060196909324
:108170003E0680933D06D3CF809165008860809352
:1081800065001092430610923E0610923D06A89597
:108190000895AC01A8958091430681114BC0909140
:1081A0006400906190936400909165009F7E90932D
:1081B00065009091640098609093640090916500D0
:1081C000977F9093650084E6849F9001859F300D92
:1081D000112480913D0690913E068217930700F589
:1081E0008091640084608093640080916500846065
:1081F0008093650087EB9BE00197F1F700C00000DA
:10820000A895809165008B7F8093650080913D06E5
:1082100090913E06019690933E0680933D06D9CFFD
:108220008091650088608093650010923E061092F0
:108230003D06A895A89581E0809343060895A895EA
:10824000682F82EE92E043D6A8950895A89582EE15
:1082500092E027D690E09DDFA8950895A895809399
:1082600042060895CF93DF9300D000D0CDB7DEB79C
:10827000809163001C821B821A821982BE016F5F8B
:108280007F4FCE01039651D18B819C8184319540E3
:1082900068F489819A81843A964040F489819A8170
:1082A0008D32914018F082E08093EB068B819C81A7
:1082B0008937954090F08B819C81843C994068F48B
:1082C00089819A81843A964040F489819A818D32DD
:1082D000914018F083E08093EB068B819C8189327A
:1082E0009A4068F089819A8184379E4040F4898160
:1082F0009A81813D974018F081E08093EB068B8155
:108300009C81863F994060F48B819C8181349640AA
:1083100038F089819A81813D974010F01092EB06E8
:108320008091EB060F900F900F900F90DF91CF91FF
:108330000895DF92EF92FF920F931F93CF93DF93F5
:10834000A89585E08093EB06DBE485E0D82E80914C
:108350004206811178C0A89585DFE0904106F12C96
:1083600003E02FE130E040E058EF62E870E080E5A4
:1083700090E00E94080C8091EB068330C1F4A89530
:1083800080914106815080934106109240061092E0
:108390003F060FE110E02CE330E046EE50E069E6E6
:1083A00070E081E090E00E94CD0A1DDEA8958091EA
:1083B000EB068230D1F4A895809141068B34A8F465
:1083C000A8958F5F809341061092400610923F0659
:1083D0000FE110E02CE330E046EE50E069E670E09B
:1083E00081E090E00E94CD0A3FDE809141068C340E
:1083F00010F0D09341068091EB0681110EC00FE181
:1084000010E02CE330E046EE50E069E670E081E0F9
:1084100090E00E94CD0A10924106C091EB06C13057
:1084200079F4A895809141060ADFA89580914106CC
:1084300090E05BDEA89510924106A895C093420695
:10844000D092EB0684CFDF91CF911F910F91FF90D7
:10845000EF90DF900895EF92FF920F931F93A895EE
:1084600082EE92E01ED58C3418F48093EA0614C094
:10847000A8951092EA0660E082EE92E028D50FE11E
:1084800010E028E230E048E550E06FEA70E080EE6E
:1084900090E00E94CD0AA8958091EA06882381F099
:1084A00082EE92E0FED4E82EF12C02E02FE130E0E3
:1084B0004FEF5FEF6AEA70E080EF90E00E94080CF7
:1084C0001F910F91FF90EF900895EF92FF920F93FD
:1084D000E090EA06F12C02E02FE130E04FEF5FEF91
:1084E0006AEA70E080EF90E00E94080C0F91FF9024
:1084F000EF900895C098AB9AAF9A8FB9779BFECF53
:108500008FB1089587E087BBC09AAB9AAF9A83E595
:108510008DB91EB880E8EEDF80E0ECDF80E0EADFB6
:108520008AE18A95F1F700C00895EF92FF920F93C8
:108530001F93CF93DF9300D000D0CDB7DEB77C017F
:108540008B01A895AB9AAF9A1C821B821A82198262
:1085500080EDD0DF80E0CEDF8FB190E09C838B8315
:108560008B819C81982F88279C838B8380E0C2DF3E
:108570002FB18B819C81822B9C838B838B819C81EF
:1085800033E0969587953A95E1F79C838B8387EC4A
:1085900090E00197F1F700C0000080E9ABDF80E0D8
:1085A000A9DF8FB190E09A83898389819A81982F7E
:1085B00088279A83898380E09DDF2FB189819A8102
:1085C000822B9A83898389819A8153E09695879536
:1085D0005A95E1F79A8389832B813C8182ED9FE054
:1085E000821B930BF7019183808389819A81F80123
:1085F000918380830F900F900F900F90DF91CF9118
:108600001F910F91FF90EF90089570D088F09F57C1
:1086100090F0B92F9927B751A0F0D1F0660F771FCE
:10862000881F991F1AF0BA95C9F712C0B13081F0AE
:1086300077D0B1E0089574C0672F782F8827B85F8E
:1086400039F0B93FCCF3869577956795B395D9F70F
:108650003EF490958095709561957F4F8F4F9F4F19
:108660000895E89409C097FB3EF490958095709525
:1086700061957F4F8F4F9F4F9923A9F0F92F96E96E
:10868000BB279395F695879577956795B795F111E3
:10869000F8CFFAF4BB0F11F460FF1BC06F5F7F4F80
:1086A0008F4F9F4F16C0882311F096E911C0772392
:1086B00021F09EE8872F762F05C0662371F096E89B
:1086C000862F70E060E02AF09A95660F771F881F6A
:1086D000DAF7880F9695879597F9089557FD905882
:1086E000440F551F59F05F3F71F04795880F97FB76
:1086F000991F61F09F3F79F0879508951216130630
:108700001406551FF2CF4695F1DF08C0161617065E
:108710001806991FF1CF8695710561050894089593
:10872000E894BB2766277727CB0197F908950BD0EC
:1087300078C069D028F06ED018F0952309F05AC09F
:108740005FC01124EECFCADFA0F3959FD1F3950F40
:1087500050E0551F629FF001729FBB27F00DB11DC5
:10876000639FAA27F00DB11DAA1F649F6627B00D55
:10877000A11D661F829F2227B00DA11D621F739F3E
:10878000B00DA11D621F839FA00D611D221F749F4C
:108790003327A00D611D231F849F600D211D822F93
:1087A000762F6A2F11249F5750408AF0E1F08823DA
:1087B0004AF0EE0FFF1FBB1F661F771F881F9150E7
:1087C0005040A9F79E3F510570F014C0AACF5F3FFB
:1087D000ECF3983EDCF3869577956795B795F7951A
:1087E000E7959F5FC1F7FE2B880F911D96958795A2
:1087F00097F9089597F99F6780E870E060E0089521
:108800009FEF80EC089500240A94161617061806A8
:108810000906089500240A94121613061406050684
:108820000895092E0394000C11F4882352F0BB0F15
:1088300040F4BF2B11F460FF04C06F5F7F4F8F4F78
:108840009F4F0895AA1BBB1B51E107C0AA1FBB1F66
:10885000A617B70710F0A61BB70B881F991F5A95CC
:10886000A9F780959095BC01CD010895EE0FFF1FEB
:108870000024001C0BBE0790F691E02D0994A29FE6
:10888000B001B39FC001A39F700D811D1124911DE4
:10889000B29F700D811D1124911D0895BB274A3090
:1088A00031F4992322F4BDE2909581959F4F01C048
:1088B000BB27FB015527AA27880F991FAA1FA417BA
:1088C00010F0A41B83955051B9F7A05DAA3308F0AE
:1088D000A95DA193009779F7B111B1931192CB01E2
:1088E00026C2CF93DF93CDB7DEB7AE014B5F5F4FAC
:1088F000FA0161917191AF018091EE069091EF06BE
:1089000003D0DF91CF9108952F923F924F925F92C3
:108910006F927F928F929F92AF92BF92CF92DF928F
:10892000EF92FF920F931F93CF93DF93CDB7DEB7F4
:108930002B970FB6F894DEBF0FBECDBF6C017B0145
:108940008A01FC0117821682838181FFBFC1CE019B
:1089500001963C01F6019381F70193FD859193FF08
:1089600081917F01882309F4ADC1853239F493FDEB
:10897000859193FF81917F01853221F4B60190E0CA
:10898000E6D1E8CF912C212C312CFFE1F315D8F062
:108990008B3279F038F4803279F08332A1F4232DD0
:1089A00020611DC08D3261F0803369F4232D216078
:1089B00016C0832D8260382EE32DE4603E2E2AC03F
:1089C000F32DF8601DC037FC2DC020ED280F2A3094
:1089D00040F08E32B9F436FC75C1232D2064322E5E
:1089E00019C036FE06C08AE0989E200D1124922EF2
:1089F00011C0EAE02E9E200D1124222EF32DF062EC
:108A00003F2E08C08C3621F4832D8068382E02C09A
:108A1000883641F4F70193FD859193FF81917F01A1
:108A20008111B3CF982F9F7D9554933028F40C5F1C
:108A30001F4F9FE399830DC0833631F0833771F068
:108A4000833509F055C020C0F801808189830E5F0D
:108A50001F4F88248394912C530112C02801F2E007
:108A60004F0E511CF801A080B18036FE03C0692D65
:108A700070E002C06FEF7FEFC5014ED14C01820163
:108A8000F32DFF773F2E15C0280122E0420E511C26
:108A9000F801A080B18036FE03C0692D70E002C0ED
:108AA0006FEF7FEFC5012DD14C01F32DF0683F2E04
:108AB000820133FC19C0822D90E088169906A0F43B
:108AC000B60180E290E043D12A94F5CFF50137FC5E
:108AD000859137FE81915F01B60190E038D1211078
:108AE0002A9421E0821A91088114910479F7E1C057
:108AF000843611F0893639F5F80137FE07C06081F8
:108B00007181828193810C5F1F4F08C060817181E8
:108B1000072E000C880B990B0E5F1F4FF32DFF766D
:108B20003F2E97FF09C090958095709561957F4F76
:108B30008F4F9F4FF0683F2E2AE030E0A30143D1D2
:108B4000882E861844C0853731F4232D2F7EB22E0F
:108B50002AE030E025C0932D997FB92E8F36C1F0E1
:108B600018F4883579F0AEC0803719F0883721F0D5
:108B7000A9C0E92FE061BE2EB4FE0DC0FB2DF4604C
:108B8000BF2E09C034FE0AC0292F2660B22E06C0AF
:108B900028E030E005C020E130E002C020E132E012
:108BA000F801B7FE07C060817181828193810C5FFB
:108BB0001F4F06C06081718180E090E00E5F1F4F03
:108BC000A30101D1882E8618FB2DFF773F2E36FE9C
:108BD0000DC0232D2E7FA22E891458F434FE0BC015
:108BE00032FC09C0832D8E7EA82E05C0B82CA32C84
:108BF00003C0B82C01C0B92CA4FE0FC0FE01E80DC3
:108C0000F11D8081803321F49A2D997EA92E09C00F
:108C1000A2FE06C0B394B39404C08A2D867809F0EE
:108C2000B394A3FC10C0A0FE06C0B21480F4280CBC
:108C3000922C9B180DC0B21458F4B60180E290E05B
:108C400086D0B394F8CFB21418F42B1802C0982C25
:108C5000212CA4FE0FC0B60180E390E078D0A2FEE4
:108C600016C0A1FC03C088E790E002C088E590E050
:108C7000B6010CC08A2D867851F0A1FE02C08BE2AD
:108C800001C080E2A7FC8DE2B60190E060D08914BB
:108C900030F4B60180E390E05AD09A94F8CF8A94E9
:108CA000F301E80DF11D8081B60190E050D08110F4
:108CB000F6CF222009F44ECEB60180E290E047D0F4
:108CC0002A94F7CFF6018681978102C08FEF9FEF3C
:108CD0002B960FB6F894DEBF0FBECDBFDF91CF91BC
:108CE0001F910F91FF90EF90DF90CF90BF90AF90CA
:108CF0009F908F907F906F905F904F903F902F90BC
:108D00000895FC010590615070400110D8F78095DE
:108D100090958E0F9F1F0895FC0161507040019047
:108D20000110D8F7809590958E0F9F1F0895DC0154
:108D3000FC01672F71917723E1F7329704C07C9192
:108D40006D9370836291AE17BF07C8F308950F93B8
:108D50001F93CF93DF93FB01238121FD03C08FEF8E
:108D60009FEF2CC022FF16C0468157812481358198
:108D70004217530744F4A081B1819D012F5F3F4FFB
:108D8000318320838C93268137812F5F3F4F378338
:108D9000268314C08B01EC01FB010084F185E02DDA
:108DA0000995892BE1F6D80116968D919C9117971C
:108DB000019617969C938E931697CE01DF91CF91D3
:108DC0001F910F910895FA01AA27283051F12031FF
:108DD00081F1E8946F936E7F6E5F7F4F8F4F9F4F4F
:108DE000AF4FB1E03ED0B4E03CD0670F781F891F91
:108DF0009A1FA11D680F791F8A1F911DA11D6A0F5F
:108E0000711D811D911DA11D20D009F468943F9111
:108E10002AE0269F11243019305D3193DEF6CF0110
:108E20000895462F4770405D4193B3E00FD0C9F7D6
:108E3000F6CF462F4F70405D4A3318F0495D31FD43
:108E40004052419302D0A9F7EACFB4E0A695979596
:108E5000879577956795BA95C9F70097610571056C
:108E600008959B01AC010A2E0694579547953795B6
:108E70002795BA95C9F7620F731F841F951FA01D10
:108E80000895DC01CB01FC01E199FECF06C0FFBBD8
:108E9000EEBBE09A31960DB20D9241505040B8F7BA
:108EA0000895E199FECF9FBB8EBBE09A99278DB3C1
:108EB0000895A8E1B0E042E050E0E5CFDC01CB014D
:108EC00002C02D9105D041505040D8F70895262F6B
:108ED000E199FECF9FBB8EBB2DBB0FB6F894E29AF3
:108EE000E19A0FBE01960895F2DF272FF1CFF89493
:028EF000FFCFB2
:108EF200140048005D0078009600B600D500F3002B
:108F020010012C01490163017C019401AC01C101F2
:108F1200D501E801010E00000002000000002A0F46
:108F22000000000044656C004F4E004F4646002092
:108F320020D1F2E0EDF6E8FF00C2E5F0F5EDE8E958
:108F420000CDE8E6EDE8E900D0F3F7EDEEE900D078
:108F5200E5E1EEEBEBE8EDE32000D1F3F8EAE00027
:108F6200ECE8EAF0EEF1F5E5EC00EFEBE0F200CA36
:108F7200E0EBE8E1F0EEE2EAE000EDE8E7E000CC69
:108F8200EEF9EDEEF1F2FC00E2E5F0F5E000C2E50B
:108F9200F0F5EDE8E920EDE0E3F02E00CDE8E6EDB6
:108FA200E8E920EDE0E3F02E20002020D0F3F7EDF9
:108FB200EEE92020200020D1F3F8EAE020EFEBE0F8
:108FC200F22000C4EEEF2E20EDE0F1F2F0EEE9EA3D
:108FD200E8002020D1F2E5EAEBEE00CAE0EBE8E19E
:108FE200F0EEE2EAE02000EDE8E7E02000C2DBD5A7
:108FF200CEC40057543D2025750A47530047533DC0
:109002002025750A534E00534E3D2025750A454EC4
:109012004400574B3D2025750A565000503D332ED3
:10902200360A5200524C3D2025750A68004F3D73A6
:10903200740A5300473D73740A530053523D5374EC
:109042006174696F6E200A57500057503D536E3657
:10905200332F506233370A57540057503D536E41F5
:10906200670A57540057503D50726F66696C6530FD
:109072000A57540057503D50726F66696C65310A49
:1090820057540057503D50726F66696C65320A57EB
:10909200540057503D50726F66696C65330A5754DD
:1090A2000057503D50726F66696C65340A57540020
:1090B20057503D50726F66696C65350A57540053BC
:1090C200523D5550686561746572200A57500053CD
:1090D200523D507265686561746572200A5750008E
:1090E20053523D4D616E75616C200A5750005352C8
:1090F2003D5265626F6C6C696E67200A575000536F
:10910200523D4368697068656174696E67200A57E9
:10911200500053523D50434268656174696E672046
:109122000A57500053523D5043200A575000C2FB89
:10913200E1E5F0E8F2E520E2FBF1EEF2F3004D3278
:1091420043726166742056352E3400202020C2F00E
:10915200E5ECFF20F0E5E1EEEBEBE8EDE3E02020CB
:10916200202000C2FBE1E5F0E8F2E520F0E5E6E8C8
:10917200EC00D2E5ECEFE5F0E0F2F3F0E020EFEE08
:10918200EBEEF7EAE8202000EDE8E7E020EFF0E878
:1091920020E4EEEDE0E3F0E5E2E500D2E5ECEFE518
:1091A200F0E0F2F3F0E020F3E2E5EBE8F7E5EDE8DA
:1091B200FF00202020202020E4EEEDE0E3F0E5E2B5
:1091C200E020202020202000C4EBE8F2E5EBFCEDBB
:1091D200EEF1F2FC20E2EFE8F2FBE2E0EDE8FF0064
:1091E200D4F3EDEAF6E8FF20E4EEEDEEE3F0E5E29B
:1091F200E000EDE8E6EDE5E3EE20EDE0E3F0E5E2A8
:10920200E0F2E5EBFF2020202000CCE0EAF1E8ECE0
:10921200E0EBFCEDE0FF20ECEEF9EDEEF1F2FC20EC
:109222002000E2E5F0F5EDE5E3EE20EDE0E3F0E528
:10923200E2E0F2E5EBFF20202000CCE0EAF1E8ECEE
:10924200E0EBFCEDE0FF20ECEEF9EDEEF1F2FC20BC
:109252002000E2E5F0F5EDE5E3EE20EDE0E3F0E5F8
:10926200E2E0F2E5EBFF20202000D2E5ECEFE5F0B2
:10927200E0F2F3F0E020E2EAEBFEF7E5EDE8FF20B2
:109282002000CAEEEDF2F0EEEBFC20EFEE20E2E57C
:10929200F0F5F320202020202000EDE8E6EDE5E3C4
:1092A200EE20EDE0E3F0E5E2E0F2E5EBFF20202046
:1092B2002000CAEEFDF4F4E8F6E8E5EDF220EFF066
:1092C200EEF4E8EBFF2020202000E2E5F0F5EDE5EA
:1092D200E3EE20EDE0E3F0E5E2E0F2E5EBFF202053
:1092E2002000CAEEFDF4F4E8F6E8E5EDF220EFF036
:1092F200EEF4E8EBFF2020202000EDE0E3F0E5E2D1
:10930200E0F2E5EBFF202000D2E5ECEFE5F0E0F241
:10931200F3F0E020EDE8E6EDE5E3EE20202020008A
:10932200EFE0E9EAE82000D2E5ECEFE5F0E0F2F365
:10933200F0E020ECE5F1F2E0202020202000C2FB4A
:10934200E1E5F0E8F2E520EFF0EEF4E8EBFC0036C0
:10935200302D393020D100CFF0EEF4E8EBFC20358F
:1093620000CFF0EEF4E8EBFC203400CFF0EEF4E8AE
:10937200EBFC203300CFF0EEF4E8EBFC203200CF20
:10938200F0EEF4E8EBFC203100CFF0EEF4E8EBFC79
:10939200203000536E416700536E506200CFF0E8F8
:1093A200EDFFF2EE202000C2DBC1D0C0D2DC00C251
:1093B200DBCACB00C2CACB00CDE0F1F2F0EEE8F29C
:1093C200FC00C7E2F3EAEEE2FBE520F1E8E3EDE0C0
:1093D200EBFB00CFF0E5E4F3F1F2E0EDEEE2EAE8D8
:1093E20000D3ECEEEBF7E0EDE8FF00C2F0E5ECFFB6
:1093F20020EFE0E9EAE80020C4E0F2F7E8EA20ED35
:10940200E8E62E20EDE0E3F0E5E2E0F2E5EBFF0036
:1094120020C4E0F2F7E8EA20ECE5F1F2E020EFE028
:04942200E9EAE8008B
:00000001FF
